:100000000C949E010C94BB010C94BB010C94BB019D
:100010000C949F090C945F090C9421040C948303A5
:100020000C946F040C9432090C94BB010C94DF08FF
:100030000C94BB010C949D050C94BB010C94E3053E
:100040000C94BB010C94BB010C94BB010C94BB0140
:100050000C94BB01303132333435363738394142B4
:10006000434445460000000306080A000003050655
:1000700007080A54000000730002631510730001A2
:100080004815117300012315207300010815217311
:100090000002B21422730002911423730001781439
:1000A000257300041D1426730004E6142773000151
:1000B000FF13307300009A155073000242135173FE
:1000C0000002C11252730001E413537300000412C2
:1000D00054730001181356730001FD125873000584
:1000E0004712807300009A1584730006B113897358
:1000F00000027E139C730001BF110000000000008D
:100100005374773D536F670D0A007374617274699D
:100110006E67204C43440D0A005645523A312E3446
:10012000390D0A0053656154616C6B3C2D3E4E6D78
:10013000656120436F6E7665727465720D0A0024E6
:100140005354414C4B2C00524D432C00474C4C2CEB
:10015000004D54572C002C4E2A002C4E2C00564C8F
:10016000572C005253412C0048444D2C0056485700
:100170002C004450542C004442542C004D57562C13
:100180000024534E4253452C005A444100484447F2
:100190000044505400534E425345005354414C4B7D
:1001A0000048444D00564857004D575600564C578E
:1001B00000444254004D54570056544700474C4C9D
:1001C00000524D4300524D42002D2D2D2D2D2D2D31
:1001D0002D2D2D20004473743A2D2D2D2D2D0044EE
:1001E00073743A0054726B3A2D2D2D2D2D005472DC
:1001F0006B3A004272673A2D2D2D2D2D0042726709
:100200003A005854453A2D2D2D2D2D005854453A7D
:1002100000546F3A20202020200046726F6D3A2053
:1002200020202020202000546F74203A2D2D2D2DC9
:100230002D2D2D00546F74203A00547269703A2DA0
:100240002D2D2D2D2D2D00547269703A00436F67AE
:100250003A2D2D2D2D2D00436F673A00436D6167B8
:100260003A2D2D2D00436D61673A0020536F673A98
:10027000202D2D2D2D0020536F673A200020546D26
:10028000703A202D2D2D2D0020546D703A20002025
:100290005744673A2D2D2D2D2D00205744673A00E5
:1002A000205753703A202D2D2D2D00205753703A92
:1002B0002000436F673A2D2D2D2D2D0020436F67B1
:1002C0003A005620004470743A2D2D2D2D2D2D000E
:1002D0004470743A0020536F673A202D2D2D2D0065
:1002E00020536F673A20005374773A2D2D2D2D2D12
:1002F00020005374773A005645523A312E34390D66
:100300000A004C697374656E696E6720204E4D4516
:1003100041004C697374656E696E67202053656196
:1003200054616C6B005374616C6B3C3D3E4E4D45AB
:1003300041204272696467650049490011241FBE6B
:10034000CFE5D8E0DEBFCDBF10E0A0E6B0E0E2EB45
:10035000F4E702C005900D92A436B107D9F713E077
:10036000A4E6B0E001C01D92A03DB107E1F70E94F4
:10037000BE2E0C944B390C940000FC0171836083F9
:100380005383428317821682158214820895CF9375
:10039000DF93EC018C819D81892BE1F08E819F811F
:1003A000E881F981E80FF91F208120930302F89476
:1003B00001969F838E836A817B818617970720F041
:1003C0000E94F4399F838E838C819D8101979D8348
:1003D0008C837894809103029927DF91CF910895BF
:1003E000FC019B018481958168177907B0F48681AF
:1003F0009781860F971F9783868362817381861703
:10040000970720F00E94F439978386838481958131
:10041000821B930B9583848308951582148208951B
:10042000FC01CB012681378162817381820F931F8A
:100430000E94F4390190F081E02DE80FF91F8081CE
:1004400099270895CF93DF93EC01462F2C813D81AE
:100450006A817B812617370718F080E090E014C08E
:10046000F8948E819F81820F931F0E94F439E88156
:10047000F981E80FF91F40838C819D8101969D834E
:100480008C8378948FEF90E0DF91CF9108950F9354
:100490001F93CF93DF938C01EB0104C0C8010E942E
:1004A0002202219668816623C9F78FEF90E0DF91E1
:1004B000CF911F910F910895FC0140E050E02481FD
:1004C0003581828193812817390710F441E050E08B
:1004D000CA010895FC0140E050E084819581860FB7
:1004E000971F228133818217930710F441E050E077
:1004F000CA010895FC01848199270895FC011582A1
:1005000014820895FC0171836083428314821382F4
:100510000895DC01FC0183818823F1F02481E22F1E
:10052000FF27EE0FFF1F8D919C911197E80FF91F88
:10053000808191819093040280930302822F8F5FC8
:10054000FD0184836281861718F00E94E839948344
:10055000FD01838181508383809103029091040285
:100560000895CF93DF93DC01EC01EC81FF27EE0FC0
:10057000FF1F8D919C91E80FF91F808191819093CD
:10058000040280930302DF91CF910895FC01862F2E
:10059000948162817727890F912D911D0E94083ADD
:1005A000880F991F0190F081E02DE80FF91F8081DD
:1005B000918190930402809303020895FC01CB0182
:1005C000248162817727820F911D0E94F439880F60
:1005D000991F0190F081E02DE80FF91F8081918132
:1005E00008950F931F93CF93DF93EC018B012B8121
:1005F0006A81261718F080E090E013C08C8177277D
:10060000820F912D911D0E94083A880F991FE88151
:10061000F981E80FF91F118300832F5F2B838FEF80
:1006200090E0DF91CF911F910F910895FC0120E0A0
:1006300030E093818281981710F421E030E0C90105
:100640000895FC01838199270895FC0120E030E0A2
:100650008381680F711D828199276817790710F4CB
:1006600021E030E0C9010895FC011382089589E07A
:1006700092E0089580916400882359F48091650088
:10068000882339F480910702882319F48FEF90E0D2
:10069000089580E090E008959C0180916400882393
:1006A00079F580916500882359F5809107028823A8
:1006B00039F580B3829586958695837080FF20C03A
:1006C0008FEF8093650020931102832F99278093E9
:1006D000080280910802813029F48CB59DB58370A1
:1006E000835F01C08DE0809306028FEF80936100ED
:1006F00089B7806189BF80E188BF8FEF90E008955E
:1007000080E090E008951F920F920FB60F9211248F
:100710002F933F938F939F93809106028B3069F4C0
:1007200080916100882349F0109260008091060258
:1007300081508093060295987BC0809106028C3090
:1007400090F080916100882371F480E1809306022B
:1007500080B3829586958695837080FF69C08FEF00
:100760008093610065C0809106028C3028F08091F2
:100770006100882309F049C080B320916000829510
:10078000869586958370992781709070332782179C
:10079000930739F0959A81E0809360008FEF809302
:1007A0006400809164008823D9F580910602882333
:1007B00091F180910602833088F08091110280FFD0
:1007C00005C081E080936000959A03C0109260009C
:1007D000959880911102869580931102809106026E
:1007E000823061F48091080280FF05C081E080932F
:1007F0006000959A03C0109260009598809106025F
:10080000813019F480936000959A8091060281509E
:10081000809306020DC089B78F7E89BF959A06C066
:1008200089B78F7E89BF959A109206021092650053
:100830009F918F913F912F910F900FBE0F901F901E
:1008400018951F920F920FB60F9211242F933F937A
:100850004F935F938F939F9346B557B52AB53BB59A
:10086000809106028C3068F080916500882349F001
:1008700080B3829586958695837080FD02C0109224
:100880006100C90196958795840F951F821793077C
:1008900010F0821B930B99BD88BD89B78F7D89BFEE
:1008A00088B7886088BF89B7886089BF8FEF8093D9
:1008B000070210921202109205029F918F915F9190
:1008C0004F913F912F910F900FBE0F901F90189551
:1008D00080916400992708951092640008951F92F2
:1008E0000F920FB60F9211242F933F934F935F9364
:1008F0006F937F938F939F93AF93BF93EF93FF93E8
:10090000809106028C3070F080916500882351F050
:1009100080B3829586958695837080FD03C0109282
:10092000610052C0809165008823B9F080B32091A6
:100930006000829586958695837099278170907066
:1009400033278217930709F43FC08FEF8093640029
:1009500081E080936000959A37C0809112028930BF
:1009600079F4869902C060E001C061E089E092E01C
:100970000E9422026091050289E092E00E94220218
:10098000809112028A3088F48091050286958093C6
:100990000502869B05C08091050280688093050250
:1009A000809112028F5F80931202809112028A302E
:1009B00059F489B7877F89BF88B7806288BF89B7B4
:1009C000806289BF10920702FF91EF91BF91AF91B2
:1009D0009F918F917F916F915F914F913F912F9157
:1009E0000F900FBE0F901F9018950F931F93CF93EA
:1009F000DF93EC0180910D0290910E02029718F4A2
:100A000080E090E014C089E092E00E94C701082FC6
:100A10001127102F00271983088389E092E00E9494
:100A2000C701080F111D198308838FEF90E0DF9134
:100A3000CF911F910F91089589B78F7E89BF89B794
:100A4000877F89BF89B78F7D89BF82E00E94360882
:100A500083E00E94360884E00E94360808954CE343
:100A600050E067E670E089E092E00E94BD010895E1
:100A700089B78F7E89BF89B78F7D89BF1092650046
:100A80001092660010921202109206020E942F0528
:100A90008D9A8E989698959A81E00E9421081FBCA5
:100AA00089E88EBD80E096E09BBD8ABD89B78062F3
:100AB00089BF88B7886388BF789408959093980118
:100AC000809397010895F3E0660F771F881F991FA1
:100AD000FA95D1F79B01AC01220F331F441F551F1C
:100AE000605070488F489F4F0E941B3A2150304001
:100AF00029B9232F332720BD089584E192E008957A
:100B00008EE192E00895982F809113028823E1F3FB
:100B10009CB91092130208951092190210921802B3
:100B200008958091180290911902892B19F48FEF82
:100B300090E0089580E090E008951F920F920FB624
:100B40000F9211242F933F934F935F936F937F9353
:100B50008F939F93AF93BF93EF93FF93CF93DF93C5
:100B6000CDB7DEB72197DEBFCDBF8BB1992783709C
:100B70009070892B21F08CB1898368E503C08CB11A
:100B80008983698184E192E00E9422022196F8948F
:100B9000DEBFCDBFDF91CF91FF91EF91BF91AF91BC
:100BA0009F918F917F916F915F914F913F912F9185
:100BB0000F900FBE0F901F901895682F8EE192E056
:100BC0000E94220208951F920F920FB60F921124D5
:100BD0002F933F934F935F936F937F938F939F9345
:100BE000AF93BF93EF93FF9380911D02882381F011
:100BF0008091220290912302892B41F08EE192E0B4
:100C00000E94C70180931C028CB905C010921D027E
:100C10008FEF80931302FF91EF91BF91AF919F915E
:100C20008F917F916F915F914F913F912F910F9095
:100C30000FBE0F901F901895CF93DF93EC0180911A
:100C4000160290911702892B71F0809118029091F1
:100C50001902892B41F084E192E00E94C701888348
:100C60008FEF90E002C080E090E0DF91CF91089597
:100C700040E550E063EA70E084E192E00E94BD014B
:100C800040EA50E065EF70E08EE192E00E94BD0125
:100C900008950E943806109298011092970188EDED
:100CA0008AB960E875E280E090E00E9463058FEF0A
:100CB0008093130210921D021092270210922602B6
:100CC000789408958091220290912302892B99F0C3
:100CD00080911D02882379F48FEF80931D028EE1AD
:100CE00092E00E94C701982F809113028823E1F3BC
:100CF0009CB910921302089590939A0180939901E0
:100D00000895E0919901F0919A01099508952F9223
:100D10003F924F925F926F927F928F929F92AF928B
:100D2000BF92CF92DF92EF92FF920F931F93CF93D8
:100D3000DF93CDB7DEB7A4970FB6F894DEBF0FBE32
:100D4000CDBF4BA32CA327013801442351F017FF3B
:100D500008C0EE24FF248701E418F50806091709E6
:100D600002C08301720169A390E02BA1211191E0DF
:100D7000E9A1E91BE150EAA318A2882E992487FC77
:100D80009094A92CB92CC801B701A50194010E9427
:100D90001B3AFB01EC5AFF4F64916F8FC801B701FA
:100DA000A50194010E941B3A69017A018EE1282E67
:100DB000312C2C0E3D1E20C0C114D104E104F104DD
:100DC000A9F0C701B601A50194010E941B3AFB01DD
:100DD000EC5AFF4F6491F1016083C701B601A50190
:100DE00094010E941B3A69017A0103C02CA1F10110
:100DF000208308942108310881010F5F1F4F8AA1C9
:100E000081508AA38F3FC1F69BA19923B9F077FE49
:100E100003C081018DE20AC04114510461047104D0
:100E200019F081018BE202C0810180E2F801808328
:100E300005C0F80181918F010E948106F9A1F1504E
:100E4000F9A3FF3FB1F7A4960FB6F894DEBF0FBE2B
:100E5000CDBFDF91CF911F910F91FF90EF90DF9069
:100E6000CF90BF90AF909F908F907F906F905F904A
:100E70004F903F902F9008952F923F924F925F9204
:100E80006F927F928F929F92AF92BF92CF92DF929A
:100E9000EF92FF920F931F93CF93DF93CDB7DEB7FF
:100EA000A4970FB6F894DEBF0FBECDBF9BA38AA355
:100EB000222E0CA336014701222351F0F7FE08C071
:100EC000EE24FF248701E618F7080809190902C073
:100ED0008401730149A380E0211081E039A0381A10
:100EE0003A9418A2A62EBB24A7FCB094CB2CDB2CE2
:100EF000C801B701A60195010E941B3AFB01EC5AFB
:100F0000FF4F64916F8FC801B701A60195010E9440
:100F10001B3A79018A019EE1492E512C4C0E5D1E2F
:100F200020C0E114F10401051105A9F0C801B701C1
:100F3000A60195010E941B3AFB01EC5AFF4F6491F8
:100F4000D2016C93C801B701A60195010E941B3A1A
:100F500079018A0103C08CA1F201808308944108C1
:100F60005108F20131963A949FEF3916D1F62220BA
:100F700099F0ADE22A1681F097FE03C0F2018DE2EE
:100F80000AC0611471048104910419F0F2018BE22A
:100F900002C0F20180E2808380E00AC02081222327
:100FA00031F08F5FAAA1BBA12D93BBA3AAA3319659
:100FB000B9A1B150B9A3BF3F89F79927A4960FB63D
:100FC000F894DEBF0FBECDBFDF91CF911F910F917F
:100FD000FF90EF90DF90CF90BF90AF909F908F9059
:100FE0007F906F905F904F903F902F90089508955D
:100FF00083B7887F856083BF12BE89B7816089BF50
:10100000109228021092290210922A0210922B02AA
:1010100008958EB5887F83608EBD1DBC1CBC89B7CA
:10102000846089BF089585B5887F846085BD14BCC0
:1010300089B7806489BF089593B7987F982B93BF31
:1010400008959EB5987F982B9EBD089595B5987F7D
:10105000982B95BD0895883040F4E82FFF27EE0FB8
:10106000FF1FE556FE4F718360830895883040F47A
:10107000E82FFF27EE0FFF1FE556FE4F118210826B
:101080000895DF92EF92FF920F931F938C01D2B6D7
:1010900010922C0210922D0210922E0210922F020A
:1010A000E3B7FF27EB59FF4FE49121E030E002C0A6
:1010B000220F331FEA95E2F7442737FD4095542F5E
:1010C00060E070E880E790E00E943D3AC8017C0152
:1010D00000271127213492E439079FE0490790E067
:1010E000590788F0CA01B90128EE33E040E050E02A
:1010F0000E941B3ACA01B901A80197010E94C9398F
:101100009B01AC010CC0CA01B901A80197010E9462
:10111000C93928EE33E040E050E00E941B3A7901E3
:101120008A01ED0CF11C011D111D20912C02309142
:101130002D0240912E0250912F0282B79927AA27A3
:10114000BB27542F432F322F2227822B932BA42BE4
:10115000B52B8E159F05A007B10738F31F910F918E
:10116000FF90EF90DF9008951092280210922902CC
:1011700010922A0210922B02089560912802709119
:10118000290280912A0290912B0208958F9A979AB2
:101190008EE685BD80E883BD89B78F7389BF12BC99
:1011A0000895982F882329F485B58F7C85BD97985D
:1011B000089585B5806285BD979A93BD08951F9265
:1011C0000F920FB60F9211242F933F934F935F937B
:1011D0006F937F938F939F93AF93BF93EF93FF93FF
:1011E0008091280290912902A0912A02B0912B02AD
:1011F0000196A11DB11D8093280290932902A0930E
:101200002A02B0932B0280912C0290912D02A09182
:101210002E02B0912F020196A11DB11D80932C02C8
:1012200090932D02A0932E02B0932F0280919B01E8
:1012300090919C01892B29F0E0919B01F0919C01F8
:101240000995FF91EF91BF91AF919F918F917F9100
:101250006F915F914F913F912F910F900FBE0F9023
:101260001F9018951F920F920FB60F9211242F9373
:101270003F934F935F936F937F938F939F93AF931E
:10128000BF93EF93FF9380919D0190919E01892BD5
:1012900029F0E0919D01F0919E010995FF91EF9158
:1012A000BF91AF919F918F917F916F915F914F917E
:1012B0003F912F910F900FBE0F901F9018951F9286
:1012C0000F920FB60F9211242F933F934F935F937A
:1012D0006F937F938F939F93AF93BF93EF93FF93FE
:1012E0008091300290913102A0913202B09133028C
:1012F0000196A11DB11D8093300290933102A093FD
:101300003202B09333028091A5019091A601892BFE
:1013100029F0E091A501F091A6010995FF91EF91C7
:10132000BF91AF919F918F917F916F915F914F91FD
:101330003F912F910F900FBE0F901F9018951F9205
:101340000F920FB60F9211242F933F934F935F93F9
:101350006F937F938F939F93AF93BF93EF93FF937D
:101360008091A7019091A801892B29F0E091A70114
:10137000F091A8010995FF91EF91BF91AF919F91D5
:101380008F917F916F915F914F913F912F910F902E
:101390000FBE0F901F90189580E090E0FC01EE0FBB
:1013A000FF1FE556FE4F118210820196883091058D
:1013B000A9F70E94F8070E9409080E941308789470
:1013C00008958091AB0199270895982F8091AB01E2
:1013D000891720F49095890F99270895891B9927DB
:1013E00008950E94BD086D317105810591053CF09D
:1013F0008091AB018F5F8093AB010E94B408089588
:1014000085E00E941C0861EF79E080E00E942B08D3
:101410000E94B4081092AB010895CF93DF93CDB72B
:10142000DEB721970FB6F894DEBF0FBECDBF982F61
:10143000198207C0000000000000000089818F5F52
:10144000898389818917B0F321960FB6F894DEBF9E
:101450000FBECDBFDF91CF9108951F93C29AC4985C
:10146000662311F4C39A01C0C3981FEF1ABB8BBB4C
:10147000C29882E30E940D0AC49A1ABA1BBBC29A90
:101480001F91089560E00E942D0A81E00E940D0ADC
:1014900008951F93162F61E00E942D0A112319F061
:1014A000812F0E940D0A1F910895CF93DF93EC01C5
:1014B00003C00E94420A219688818823D1F7DF91D8
:1014C000CF910895CF93DF93EC0103C00E94420AAD
:1014D0002196FE0184918823C9F7DF91CF91089569
:1014E00063E080580E94490A089563E081E00E9409
:1014F000490A8AEF0E940D0A8AEF0E940D0A8AEFBC
:101500000E940D0A8AEF0E940D0A0895613039F099
:10151000613050F0623029F0633031F404C0805EF5
:1015200003C0805C01C0805A63E080680E94490A61
:1015300008951F931FEF17BBC19884EF91E00E949D
:10154000410882E088BB84EF91E00E9441081ABA0A
:101550001BBB63E084E30E94490A63E089E00E94C8
:10156000490A63E080E30E94490A63E08CE00E943C
:10157000490A63E081E00E94490A63E086E00E9434
:10158000490A1F91089508950895089508951F9395
:10159000CF93DF93AC018091B501882339F48FEFAD
:1015A0008093B5011092B7011092B6014F3F5105DB
:1015B00029F020F01092B7011092B6018091B60187
:1015C0009091B7018130910509F456C081309105A1
:1015D00040F08230910509F46CC0039709F09EC079
:1015E00080C04F3F510509F008F498C01092B20135
:1015F0004093B40146E050E066E770E08CEA91E089
:101600000E944D39CCEAD1E019C09091AC01809193
:10161000B401981719F481E090E046C06091B201DE
:101620006F5F6093B20186E0689FB00111246A5831
:101630007F4F46E050E0CE010E944D398091AD01D0
:101640009091AE01892B09F78091DA02882309F481
:1016500065C081E090E09093B7018093B6018091DE
:10166000B4018093AC011092AE011092AD011092C2
:10167000B1011092B00152C08091DA02882329F0A2
:10168000842F8F708093AF0109C09A012F70307042
:101690008091AF01992728173907E1F51092B3011E
:1016A0004093B80182E090E09093B7018093B60137
:1016B00035C08091B3018F5F8093B3019927FC01FE
:1016C000E854FE4F40832091AF0133272F5F3F4FF7
:1016D0008217930719F583E090E09093B701809308
:1016E000B601E091B001F091B101309719F088EBAB
:1016F00091E00995A0E0B0E00E94A339802D8823F5
:1017000049F01091AC010E94800548EB51E0612F37
:101710000E9442161092B7011092B601DF91CF914C
:101720001F910895089564E070E087E892E00E94B8
:101730002503882339F166E571E087E892E00E948D
:10174000F10260915603772784E0660F771F8A9530
:10175000E1F76F5F7F4F87E892E00E94F1026091AE
:101760005703772787E892E00E94F10260915503C2
:10177000772787E892E00E94F102809154038F7EE0
:101780008093540308950F931F9364E070E087E8FB
:1017900092E00E942503882399F1009150031127BC
:1017A00026E0000F111F2A95E1F780915103080FE1
:1017B000111D64E571E087E892E00E94F102602F5C
:1017C0006295607F77276F5F7F4F87E892E00E9486
:1017D000F10294E0169507959A95E1F71127B80163
:1017E00087E892E00E94F10260914F03772787E833
:1017F00092E00E94F10280914E038F7E80934E030F
:101800001F910F91089565E070E087E892E00E94D3
:101810002503882309F452C069E871E087E892E063
:101820000E94F10220911C0330911D03C9016AE559
:1018300070E00E94F439E4E0660F771FEA95E1F763
:10184000217030703695322F222737952795260F35
:10185000371F2E5F622F772787E892E00E94F10200
:1018600020911C0330911D03C9016AE570E00E94BC
:10187000F4398AE590E0AC01649FC001659F900D4A
:10188000749F900D1124281B390B3695279533270B
:10189000B90187E892E00E94F10260E070E087E819
:1018A00092E00E94F10260E270E087E892E00E941C
:1018B000F10280911E038F7E80931E0380E090E0F2
:1018C00008951F93CF93DF9367E070E087E892E07D
:1018D0000E942503882349F162EA71E087E892E0DB
:1018E0000E94F10280915A03992781FF03C064E4AA
:1018F00070E007C082FF03C064E270E002C064E0F1
:1019000070E087E892E00E94F10210E0C7E8D2E0C0
:1019100060E070E0CE010E94F1021F5F1530C1F758
:1019200080915B038F7E80935B0380E090E0DF918A
:10193000CF911F9108951F9369E070E087E892E0CE
:101940000E942503882309F480C062E871E087E8DB
:1019500092E00E94F10265E070E087E892E00E9468
:10196000F10280916403882311F48BE201C080535B
:1019700060916503662319F4182F105406C0162FC2
:101980001295110F110F107C180F612F772787E820
:1019900092E00E94F1021095612F772787E892E08C
:1019A0000E94F10280916503882311F48AE008C047
:1019B0009927C0978C7F9070959587959595879579
:1019C00060916603662319F4182F105504C0162F72
:1019D0001295107F180F612F772787E892E00E94F9
:1019E000F1021095612F772787E892E00E94F102BB
:1019F00080916603882311F482E009C09927C0977B
:101A000080739070F4E095958795FA95E1F7609171
:101A10006703662319F4182F145505C0162F1053A9
:101A2000110F110F180F612F772787E892E00E949E
:101A3000F1021095612F772787E892E00E94F1026A
:101A4000809176038F7E8093760380E090E01F91F3
:101A500008950F931F93CF93DF9369E070E087E8B9
:101A600092E00E942503882309F4ECC065E871E048
:101A700087E892E00E94F10260910A036295607F1C
:101A80006A5F772787E892E00E94F10260910A037B
:101A900070910B0384E0769567958A95E1F7772737
:101AA00087E892E00E94F102E0911603F09117039B
:101AB000CF0164E873E00E94F4399B01462F55275B
:101AC00084E893E0BC01469FC001479F900D569F5C
:101AD000900D1124E81BF90BCF0165E070E00E9426
:101AE000F439EB01CB018295807F682F620F8091E2
:101AF0001B038111685F772787E892E00E94F1025B
:101B000004E0D695C7950A95E1F7BE016F70062FE0
:101B100060910F0370911003809111039091120353
:101B2000683E23E0720720E0820720E0920790F0F1
:101B3000653C2FE9720720E0820720E0920718F049
:101B40002AEF3FE008C02AE030E040E050E00E9489
:101B50001B3A01C0262F2295207F200F622F772766
:101B600087E892E00E94F10260910F0370911003E8
:101B70008091110390911203683E23E0720720E0E8
:101B8000820720E09207C0F0653C2FE9720720E051
:101B9000820720E0920710F02FEF16C02AE030E015
:101BA00040E050E00E941B3A14E056954795379567
:101BB00027951A95D1F708C0B4E096958795779543
:101BC0006795BA95D1F7262F622F772787E892E09D
:101BD0000E94F10280910F0390911003A0911103D4
:101BE000B0911203885E9340A040B04010F400E131
:101BF00001C000E080910403823509F4005C095FB4
:101C0000602F772787E892E00E94F10260E070E0A1
:101C100087E892E00E94F10200951127B80187E859
:101C200092E00E94F10280910C038F7E80930C035E
:101C3000809118038F7E80931803809113038F7E09
:101C40008093130380E090E0DF91CF911F910F917B
:101C5000089563E070E087E892E00E9425038823FE
:101C600009F44DC063E571E087E892E00E94F1025B
:101C70002091050330910603C9016AE070E00E94DB
:101C8000F439CB016AE570E00E94F439FB01C90127
:101C900065E070E00E94F43963707070660F660F43
:101CA0006E0F6295607F772787E892E00E94F102CD
:101CB00080910503909106036AE070E00E94F43978
:101CC0009B01CB016AE570E00E94F4398AE590E05F
:101CD000AC01649FC001659F900D749F900D11240D
:101CE000281B2695622F77276F73707087E892E024
:101CF0000E94F102809107038F7E8093070308956D
:101D000064E070E087E892E00E942503882321F1D7
:101D100060E271E087E892E00E94F10261E070E029
:101D200087E892E00E94F1026091E3027091E40280
:101D3000707087E892E00E94F1026091E302709176
:101D4000E402672F772787E892E00E94F1028091F2
:101D5000E502877E8093E502089564E070E087E8FD
:101D600092E00E942503882321F162E571E087E873
:101D700092E00E94F10261E070E087E892E00E9448
:101D8000F1026091E8027091E902707087E892E0D8
:101D90000E94F1026091E8027091E902672F7727B3
:101DA00087E892E00E94F1028091EA028F7E8093A0
:101DB000EA020895CF93DF9365E070E087E892E050
:101DC0000E9425038823B9F161E571E087E892E07C
:101DD0000E94F10262EA70E087E892E00E94F1025C
:101DE0006091FB02772787E892E00E94F1029091D0
:101DF000FF0284E6989FB001112480910003680FD0
:101E0000711D80910203853419F4EB01D06802C082
:101E1000EB01DF776C2F772787E892E00E94F102D1
:101E20006D2F772787E892E00E94F1028091FC02F3
:101E30008F7E8093FC02DF91CF910895CF93DF9343
:101E400065E070E087E892E00E9425038823B9F1FD
:101E500060E571E087E892E00E94F10262EA70E0DA
:101E600087E892E00E94F1026091F502772787E807
:101E700092E00E94F1029091F90284E6989FB001ED
:101E800011248091FA02680F711D8091010383353E
:101E900019F4EB01D06802C0EB01DF776C2F7727D4
:101EA00087E892E00E94F1026D2F772787E892E0A1
:101EB0000E94F1028091F6028F7E8093F602DF91FC
:101EC000CF9108950F931F9364E070E087E892E04C
:101ED0000E942503882321F10091260310912703F6
:101EE0000C591F4F67E271E087E892E00E94F1020F
:101EF00061E070E087E892E00E94F102602F7727AE
:101F000087E892E00E94F102012F1127B80187E8CB
:101F100092E00E94F102809128038F7E8093280333
:101F20001F910F91089564E070E087E892E00E94AD
:101F300025038823D9F161E171E087E892E00E94EE
:101F4000F10261E070E087E892E00E94F102809186
:101F500086022091320330913303882341F0C90176
:101F60006AE070E00E94F4396058772708C0C90120
:101F70006AE070E00E94F43977276F77707087E825
:101F800092E00E94F10280913203909133036AE063
:101F900070E00E94F4399927BC0187E892E00E9422
:101FA000F102809134038F7E80933403089564E0BE
:101FB00070E087E892E00E942503882321F160E128
:101FC00071E087E892E00E94F10261E070E087E84A
:101FD00092E00E94F10260912D0370912E03672F11
:101FE000772787E892E00E94F10260912D037091BB
:101FF0002E03707087E892E00E94F10280912F0317
:102000008F7E80932F03089565E070E087E892E06B
:102010000E942503882361F160E071E087E892E087
:102020000E94F10262E070E087E892E00E94F10213
:102030008091EF02882319F060E470E002C060E054
:1020400070E087E892E00E94F1026091ED0277274C
:1020500087E892E00E94F1026091EE02772787E81C
:1020600092E00E94F1028091F2028F7E8093F20250
:10207000089563E070E087E892E00E9425038823DA
:10208000D1F060E371E087E892E00E94F10260E045
:1020900070E087E892E00E94F10260912B037727BD
:1020A0006F70707087E892E00E94F10280912C03BB
:1020B0008F7E80932C030895EF92FF921F93CF930E
:1020C000DF93EC01162F662349F480E090E00EC008
:1020D00069917991C7010E94F10204C0F7E8EF2EDF
:1020E000F2E0FF2E1150A0F78FEF90E0DF91CF913B
:1020F0001F91FF90EF90089580913B0384FF6BC088
:1021000067E070E087E892E00E942503882309F4E5
:1021100062C065E271E087E892E00E94F10260919E
:102120003C0370913D0380913E0390913F032FEF5C
:102130003FEF40E050E00E941B3A2295207F2C5F49
:10214000622F772787E892E00E94F10260913C03BA
:10215000772787E892E00E94F10260913C0370913A
:102160003D0380913E0390913F03672F782F892F85
:102170009927772787E892E00E94F1026091370360
:10218000772787E892E00E94F1026091370370910F
:1021900038038091390390913A03672F782F892F64
:1021A0009927772787E892E00E94F102609139032E
:1021B000772787E892E00E94F102809140038F7EAA
:1021C0008093400380913B038F7E80933B030E946A
:1021D000E1098093420308958091DB02882309F48A
:1021E000CDC08091F202992784FF05C086FD03C00F
:1021F0000E94041008958091EA02992784FF09C083
:1022000086FD07C08091D402882319F00E94AD0E8C
:1022100008958091E502282F3327C90188719070B5
:10222000892B29F026FD03C00E94800E089580911D
:102230003B03992784FF05C086FD03C00E947C10E4
:10224000089580912803992784FF05C086FD03C067
:102250000E94620F08958091E0028823E9F0809146
:10226000F602282F332724FF08C08091030384FD42
:1022700004C026FD02C00E941E0F8091FC02282F80
:10228000332724FF09C08091030384FD05C026FD88
:1022900003C00E94DA0E089580913403992784FFC9
:1022A00005C086FD03C00E94930F089580912F03FF
:1022B000992784FF05C086FD03C00E94D70F0895AB
:1022C00080912C0384FF0AC0ACE0B0E00E94A339E7
:1022D000802D882319F00E943910089580910703FA
:1022E000992784FF05C086FD03C00E94290E08952A
:1022F00080911E03282F3327C90188719070892B84
:1023000029F026FD03C00E94030C089580914E031E
:10231000992784FF05C086FD03C00E94C30B089562
:1023200080915403992784FF05C086FD03C00E9455
:10233000930B089580910C03282F332724FF0CC0A2
:102340008091180384FF08C08091130384FF04C0A8
:1023500026FD02C00E94290D80917603992784FFF3
:1023600004C086FD02C00E949B0C80915B039927EC
:1023700084FF04C086FD02C00E94610C08950F9383
:102380001F938C01FC01808182958F709927AC018D
:10239000437050702DE230E0B901469F9001479F95
:1023A000300D569F300D112441814F73240F311D84
:1023B000220F331F8C70907068E070E00E94083A22
:1023C000260F371F30931D0320931C0380911E039B
:1023D000816C80931E030E94E10980932003809109
:1023E000E20281688093E202F801828180934A03CD
:1023F00080914B03816C80934B030E94E109809391
:102400004D031F910F910895FC015091070355FD55
:102410003DC04081842F82958F7099278370907082
:102420002AE530E0B901869F9001879F300D969F85
:10243000300D1124818199278F739070880F991F17
:10244000280F391F842F881F8827881F280F311DC8
:10245000C90173E0880F991F7A95E1F7220F331FA6
:10246000280F391F4A7011F02B5F3F4F309306033E
:1024700020930503516C509307030E94E109809358
:1024800009038091E20281688093E2020895CF936C
:10249000DF93EC014091F60245FD70C08981809385
:1024A000F5028A819927982F88272B81820F911D09
:1024B0006AE070E00E94F4399B01CB0164E670E0B1
:1024C0000E94F4396093F90284E690E0FC016E9F6B
:1024D000C0016F9F900D7E9F900D1124281B2093AB
:1024E000FA02888184FF02C083E501C08EE48093F4
:1024F0000103416C4093F6020E94E1098093F802C7
:102500008091E20281688093E2028C818093FB02D9
:102510008D819927982F88272E81820F911D6AE03F
:1025200070E00E94F4399B01CB0164E670E00E94E8
:10253000F4396093FF0284E690E0AC01649FC0012F
:10254000659F900D749F900D1124281B209300030C
:10255000888185FF02C085E401C087E5809302037E
:102560008091FC02816C8093FC020E94E1098093BF
:10257000FE028091E20281688093E202DF91CF91B6
:1025800008951F93FC011091FC0215FD34C0818158
:102590008093FB024381242F33272F773070322F13
:1025A00022278281280F311DC90164E670E00E9454
:1025B000F4396093FF0284E690E0FC016E9FC00155
:1025C0006F9F900D7E9F900D1124281B2093000378
:1025D00047FF02C085E401C087E580930203116CC8
:1025E0001093FC020E94E1098093FE028091E202B6
:1025F00081688093E2021F910895FC01828180939B
:102600005503808182958F708093560381818093DA
:10261000570380915403816C809354030E94E10915
:10262000809359038091E20281688093E2020895C9
:10263000FC018181992724E0880F991F2A95E1F7F1
:10264000208122952F70820F911D228120934F03AC
:102650009C0196E0369527959A95E1F720935003D3
:102660008F738093510380914E03816C80934E034E
:102670000E94E109809353038091E2028168809374
:10268000E20208951F93FC011091F60215FD34C07B
:1026900081818093F5024381242F33272F77307077
:1026A000322F22278281280F311DC90164E670E094
:1026B0000E94F4396093F90284E690E0FC016E9F79
:1026C000C0016F9F900D7E9F900D1124281B2093B9
:1026D000FA0247FF02C083E501C08EE48093010344
:1026E000116C1093F6020E94E1098093F802809128
:1026F000E20281688093E2021F910895FC018081CB
:1027000082958F709927AC01437050702DE230E0B4
:10271000B901469F9001479F300D569F300D1124FF
:1027200041814F73240F311D220F331F8C70907025
:1027300068E070E00E94083A260F371F30931D03AF
:1027400020931C0380911E03816C80931E030E94C2
:10275000E109809320038091E20281688093E20284
:102760000895FC01808182958F709927AC01437098
:1027700050702DE230E0B901469F9001479F300D27
:10278000569F300D112441814F73240F311D220FAC
:10279000331F8C70907068E070E00E94083A260F3A
:1027A000371F30931D0320931C0380911E03816CFF
:1027B00080931E030E94E109809320038091E2022E
:1027C00081688093E2020895FC0182819927982F05
:1027D00088272181820F911D9093E9028093E8025E
:1027E0008091EA02816C8093EA028091E202816822
:1027F0008093E2020E94E1098093EC020895FC01BB
:10280000218133272456304082819927982F8827A9
:10281000280F391F30932703209326038091280324
:10282000816C809328030E94E10980932A038091A0
:10283000E20281688093E2020895FC01228133273D
:1028400044275527542F432F322F222780818295EA
:102850008F709927AA27BB27DC0199278827280F83
:10286000391F4A1F5B1F8181280F311D411D511DDA
:1028700020933C0330933D0340933E0350933F032A
:102880002481332744275527542F432F322F2227C3
:102890008381280F311D411D511D85819927AA274C
:1028A000BB278F709070A070B070DC0199278827CB
:1028B000280F391F4A1F5B1F2093370330933803BB
:1028C0004093390350933A0380914003816C809385
:1028D000400380913B03816C80933B030E94E1099C
:1028E000809342038091E20281688093E20208951E
:1028F000FC0181812AE0829FC0011124909327036B
:102900008093260380912803816C809328030E9482
:10291000E10980932A038091E20281688093E202B8
:102920000895FC0182819927982F88272181820FA1
:10293000911DAA27BB2780933C0390933D03A0934E
:102940003E03B0933F0380914003816C809340032A
:102950000E94E109809342038091E20281688093A2
:10296000E2020895FC012281332744275527542F82
:10297000432F322F22278181280F311D411D511DE8
:1029800083819927AA27BB278F709070A070B070A1
:10299000DC0199278827280F391F4A1F5B1F2093C6
:1029A0003703309338034093390350933A038091AF
:1029B0003B03816C80933B030E94E10980934203B7
:1029C0008091E20281688093E2020895FC01858192
:1029D00086FF1DC082819927982F88272181820F29
:1029E000911D6AE070E00E94F4397093E4026093F4
:1029F000E3028091E502816C8093E5028091E2021E
:102A000081688093E2020E94E1098093E7020895C1
:102A1000FC0182819927982F88272181820F911D9F
:102A20009093E4028093E3028091E502816C8093AD
:102A3000E5028091E20281688093E2020E94E1094E
:102A40008093E7020895FC01818199278F77907028
:102A50009C0153E0220F331F5A95E1F7880F991F0D
:102A6000820F931F2281820F911D909333038093D5
:102A7000320380913403816C809334038091E202AD
:102A800081688093E2020E94E109809336030895F1
:102A9000FC0181819927982F88272281820F911D1F
:102AA00090932E0380932D0380912F03816C80934C
:102AB0002F038091E20281688093E2020E94E10983
:102AC000809331030895FC01818199278F70907064
:102AD0008130910551F48091CE039091CF038160B4
:102AE0009093CF038093CE0302C0049711F18381AA
:102AF0009927982F88272281820F911D9093EE02AB
:102B00008093ED028091F202816C8093F2020E9428
:102B1000E1098093F4028091E20281688093E202ED
:102B20008091CE039091CF038D7F9093CF038093BC
:102B3000CE030895FC01918190932B0380912C0387
:102B4000816C80932C038091E20281688093E20281
:102B5000992341F084E1989F802D11240E94D1088F
:102B6000979A089580E00E94D10897980895DC0113
:102B7000FB018C918C3219F48DE28193108280E0FC
:102B800003C021938F5F11962C912C3221F02223C8
:102B900011F08417B1F71082282F02C011922F5F15
:102BA0002417E0F302C011968F5F2C912C3231F084
:102BB000222321F02D3011F02A30A9F7992708950A
:102BC000CF93DF93FB0120E030E004C0119211921B
:102BD0002F5F3F4F24173507CCF3FB019183808390
:102BE000EC0181E090E019C028812D30C9F02E3031
:102BF00028F42223A9F02A3079F412C02A3281F075
:102C00002C3251F4DE011D92FC01EE0FFF1FE60F86
:102C1000F71FB183A083019621968417950724F3AB
:102C2000DF91CF910895FC018081843209F43196BF
:102C300080E002C0822731962081222331F02A329F
:102C400021F02D3011F02A30A9F799270895FC01C1
:102C5000AC014F5F5F4F8181882311F420E009C0F0
:102C60008081282F20532A3008F027502295207F7A
:102C7000FA019081892F80538A3008F08750820FA3
:102C8000992708956F927F928F929F92AF92BF92F1
:102C9000CF92DF92EF92FF920F931F93CF93DF9328
:102CA0003C01C62EEA018091C801882309F05FC06B
:102CB00018811F701E5F63E0169FB001112412502F
:102CC000625F7F4FC3010E946A02882309F44FC0EC
:102CD0006FE371E084E392E00E945639DD24EE2434
:102CE000FF2400E320E042E060E18BE392E00E94F9
:102CF0003C07E82FFF27E55CFD4F21961F5F4E0143
:102D0000810E911C21978CE281935F01C990DD2493
:102D1000EE24FF2400E320E042E060E1CF010E94C6
:102D20003C07F501E80FF11DC815D90561F78AE2E6
:102D300081935F0185E392E00E9413169927AA27E9
:102D4000BB276C017D0120E042E060E1C5010E94EB
:102D50003C07A80EB11CF5018DE081938AE0E501E6
:102D60008983118264E372E0C3010E944702DF910C
:102D7000CF911F910F91FF90EF90DF90CF90BF9078
:102D8000AF909F908F907F906F9008954F925F9239
:102D90007F928F929F92AF92BF92CF92DF92EF92EB
:102DA000FF920F931F93CF93DF932C016CE370E09E
:102DB0000E946A02882309F483C166ED72E084E30D
:102DC00092E00E946B3967E471E087E392E00E9431
:102DD000563980914E0380FD03C0EBE3F2E02EC034
:102DE000C0904F03DD24EE24FF2400E320E042E006
:102DF0006AE08BE392E00E943C07A82EBB248BE3A1
:102E000092E0A80EB91EC0905003DD24EE24FF24EA
:102E100020E042E06AE0C5010E943C07A80EB11C18
:102E2000C0905103DD24EE24FF2420E042E06AE05C
:102E3000C5010E943C07F501E80FF11D1CE2DF010E
:102E40001D934D0181E48183ED011983E2E0F0E0FF
:102E50008E0E9F1EC090F502DD24EE24FF2400E3B9
:102E600020E042E06AE0C4010E943C07880E911C09
:102E7000C090F902DD24EE24FF2420E042E06AE065
:102E8000C4010E943C07880E911C3EE2732ED401BF
:102E90007D924D01C090FA02DD24EE24FF2420E053
:102EA00042E06AE0CD010E943C07880E911CE401DB
:102EB00019935E0180910103F4018183198382E0FB
:102EC00090E0A80EB91EC090FB02DD24EE24FF2482
:102ED00020E043E06AE0C5010E943C07A80EB11C57
:102EE000C090FF02DD24EE24FF2420E042E06AE0EF
:102EF000C5010E943C07A80EB11CD5017D925D0161
:102F0000C0900003DD24EE24FF2420E042E06AE0CC
:102F1000CD010E943C07A80EB11CF50111938091D0
:102F20000203E50189831183EF0122968091EA0271
:102F300080FF2DC08091E8029091E9026AE070E084
:102F40000E94F439882799276B017C0120E043E037
:102F50006AE0CE010E943C075E01A80EB11CF5019B
:102F600071925F018091E8029091E9026AE070E05D
:102F70000E94F439AA27BB276C017D0120E041E0C3
:102F80006AE0CF010E943C07E501C80FD11D1993EB
:102F90008091070380FF33C0809105039091060361
:102FA0006AE070E00E94F439882799276B017C0160
:102FB00000E320E043E06AE0CE010E943C075E01AE
:102FC000A80EB11CD5017D925D0180910503909101
:102FD00006036AE070E00E94F439AA27BB276C015F
:102FE0007D0120E041E06AE0C5010E943C07E50167
:102FF000C80FD11D809107038E7F8093070319931B
:103000008091540380FF2AC0C0905703DD24EE2432
:10301000FF2400E320E042E06AE0CE010E943C078A
:103020005E01A80EB11CC0905603DD24EE24FF24DF
:1030300020E042E06AE0C5010E943C07A80EB11CF6
:10304000C0905503DD24EE24FF2420E042E06AE036
:10305000C5010E943C07E501C80FD11DFE01119377
:103060005F0119838AE2818382E090E0A80EB91E95
:1030700085E392E00E9413169927AA27BB276C01CB
:103080007D0100E320E042E060E1C5010E943C07D1
:10309000A80EB11CF5018DE081938AE0E5018983DA
:1030A000118264E372E0C2010E9447028091FC0237
:1030B0008E7F8093FC028091F6028E7F8093F602D1
:1030C000DF91CF911F910F91FF90EF90DF90CF9004
:1030D000BF90AF909F908F907F905F904F9008959A
:1030E0005F926F927F928F929F92AF92BF92CF9298
:1030F000DF92EF92FF920F931F93CF93DF933C01E8
:103100006CE370E00E946A02882309F4E4C066ED73
:1031100072E084E392E00E946B396CE471E087E333
:1031200092E00E945639C090F502DD24EE24FF247F
:1031300000E320E042E06AE08BE392E00E943C077B
:10314000882E99248BE392E0880E991EC090F90294
:10315000DD24EE24FF2420E042E06AE0C4010E9466
:103160003C07880E911C5EE2552EE40159924E01F7
:10317000C090FA02DD24EE24FF2420E042E06AE061
:10318000CE010E943C07880E911C1CE2F4011193B1
:103190005F0180910103E40189831183E2E0F0E0A3
:1031A000AE0EBF1EC090FB02DD24EE24FF2420E003
:1031B00043E06AE0C5010E943C07A80EB11CC09024
:1031C000FF02DD24EE24FF2420E042E06AE0C50196
:1031D0000E943C07A80EB11CE50159925E01C09007
:1031E0000003DD24EE24FF2420E042E06AE0CE016B
:1031F0000E943C07A80EB11CF501119380910203B7
:10320000E50189831183EF01229680914E0380FFAF
:1032100029C0C0904F03DD24EE24FF2420E042E0CB
:103220006AE0CE010E943C075E01A80EB11CC0906E
:103230005003DD24EE24FF2420E042E06AE0C501D3
:103240000E943C07A80EB11CC0905103DD24EE245F
:10325000FF2420E042E06AE0C5010E943C07E5014E
:10326000C80FD11DFE01119380910303882311F033
:1032700086E501C081E489838AE2818342E0A42E4D
:10328000B12CAE0EBF1E85E392E00E941316992763
:10329000AA27BB276C017D0100E320E042E060E14A
:1032A000C5010E943C07A80EB11CF5018DE0819379
:1032B0008AE0E5018983118264E372E0C3010E9420
:1032C00047028091FC028E7F8093FC028091F6027F
:1032D0008E7F8093F602DF91CF911F910F91FF9027
:1032E000EF90DF90CF90BF90AF909F908F907F90A6
:1032F0006F905F9008956F927F928F929F92AF929E
:10330000BF92CF92DF92EF92FF920F93CF93DF9312
:103310003C0163E170E00E946A02882309F46FC0F7
:1033200066ED72E084E392E00E946B3961E571E042
:1033300087E392E00E9456398091260390912703FB
:103340006AE070E00E94F439882799276B017C01BC
:1033500000E320E043E06AE08BE392E00E943C0758
:10336000A82EBB248BE392E0A80EB91E8EE2E501E5
:1033700089935E0180912603909127036AE070E0B3
:103380000E94F439AA27BB276C017D0100E020E0F0
:1033900041E06AE0CE010E943C07A80EB11C8CE21D
:1033A000F50181934F0183E4E50189838AE28183FA
:1033B000E2E0F0E08E0E9F1E85E392E00E9413167D
:1033C0009927AA27BB276C017D0100E320E042E09A
:1033D00060E1C4010E943C07880E911CF4018DE05D
:1033E00081938AE0E4018983118264E372E0C3017E
:1033F0000E944702809128038E7F80932803DF91EB
:10340000CF910F91FF90EF90DF90CF90BF90AF9052
:103410009F908F907F906F9008958F929F92AF9220
:10342000BF92CF92DF92EF92FF920F93CF93DF93F1
:103430004C016FE170E00E946A02882309F4BFC06A
:1034400066ED72E084E392E00E946B396EE571E014
:1034500087E392E00E94563980914003882319F453
:10346000CBE3D2E039C060913C0370913D03809181
:103470003E0390913F032AE030E040E050E00E949C
:103480001B3A69017A0100E320E045E06AE08BE342
:1034900092E00E943C07A82EBB248BE392E0A80E8A
:1034A000B91E8EE2E501899360913C0370913D0362
:1034B00080913E0390913F032AE030E040E050E0ED
:1034C0000E941B3A6B017C0120E041E06AE0CE01E2
:1034D0000E943C07C80FD11D6AE571E0CE010E9431
:1034E0005639239680913B038823B9F160913703C5
:1034F000709138038091390390913A0324E630E0CB
:1035000040E050E00E941B3A69017A0100E320E0AC
:1035100044E06AE0CE010E943C075E01A80EB11CA7
:103520008EE2F50181935F0160913703709138035A
:103530008091390390913A0324E630E040E050E076
:103540000E941B3A6B017C0120E042E06AE0C50169
:103550000E943C07E501C80FD11D66E571E0CE0170
:103560000E94563963E0A62EB12CAC0EBD1E85E339
:1035700092E00E9413169927AA27BB276C017D01B0
:1035800000E320E042E060E1C5010E943C07A80E94
:10359000B11CF5018DE081938AE0E50189831182F8
:1035A00064E372E0C4010E94470280913B038E7F76
:1035B00080933B03809140038E7F80934003DF9193
:1035C000CF910F91FF90EF90DF90CF90BF90AF9091
:1035D0009F908F9008958F929F92AF92BF92CF92BB
:1035E000DF92EF92FF920F93CF93DF934C0165E14F
:1035F00070E00E946A02882309F463C066ED72E0FD
:1036000084E392E00E946B3963E671E087E392E025
:103610000E945639C0904A03C7FC03C0CBE3D2E0F6
:1036200005C08DE280933B02CCE3D2E0DD24C7FCF1
:10363000D094ED2CFD2C00E32DE244E06AE0CE01B5
:103640000E943C07DE01A80FB11D9CE2FD01919391
:1036500081E4ED018983DF0111969183FD013196AB
:10366000ED0199835F010894A11CB11C86E581835B
:103670008AE2F501818382E090E0A80EB91E85E31D
:1036800092E00E9413169927AA27BB276C017D019F
:1036900020E042E060E1C5010E943C07A80EB11C99
:1036A000F5018DE081938AE0E5018983118264E36D
:1036B00072E0C4010E94470280914B038E7F809389
:1036C0004B03DF91CF910F91FF90EF90DF90CF9060
:1036D000BF90AF909F908F9008958F929F92AF92DE
:1036E000BF92CF92DF92EF92FF920F93CF93DF932F
:1036F0004C0161E170E00E946A02882309F44DC028
:1037000066ED72E084E392E00E946B3968E671E056
:1037100087E392E00E945639C0901C03D0901D03AD
:10372000EE24FF2400E320E043E06AE08BE392E034
:103730000E943C07E82FFF27E55CFD4F8CE2DF018C
:103740008D935D018DE481838AE2ED018983E2E05E
:10375000F0E0AE0EBF1E85E392E00E94131699279B
:10376000AA27BB276C017D0120E042E060E1C50192
:103770000E943C07A80EB11CF5018DE081938AE000
:10378000E5018983118264E372E0C4010E9447026B
:1037900080911E038E7F80931E03DF91CF910F9146
:1037A000FF90EF90DF90CF90BF90AF909F908F9061
:1037B00008954F925F926F927F928F929F92AF92F5
:1037C000BF92CF92DF92EF92FF920F931F93CF930E
:1037D000DF932C016AE270E00E946A02882309F4F8
:1037E00027C166ED72E084E392E00E946B396DE6DA
:1037F00071E087E392E00E94563980910703992790
:103800008F779070892B19F4ABE3B2E033C08091CD
:103810000503909106036AE070E00E94F43988275E
:1038200099276B017C0100E320E043E06AE08BE331
:1038300092E00E943C07A82EBB244BE352E0A40E6A
:10384000B51E8EE2E50189938091050390910603F0
:103850006AE070E00E94F439AA27BB276C017D0161
:1038600000E020E041E06AE0CE010E943C07DE017A
:10387000A80FB11D1CE2FD01119384E5ED018983C0
:103880001183EF01229680911E0399278F77907004
:10389000892B79F0C0901C03D0901D03EE24FF24E7
:1038A00000E320E043E06AE0CE010E943C07C80F3D
:1038B000D11DFE0111938DE489831183EF012296BE
:1038C0008091E50299278F779070892B81F1809103
:1038D000E3029091E4026AE070E00E94F4398827E4
:1038E00099276B017C0100E320E043E06AE0CE0110
:1038F0000E943C075E01A80EB11C8EE2F501819387
:103900005F018091E3029091E4026AE070E00E941E
:10391000F439AA27BB276C017D0100E020E041E0DB
:103920006AE0CF010E943C07E501C80FD11DFE01EE
:1039300011938EE489831183EF0122968091E50231
:1039400099278F779070892B09F43FC02091E3026B
:103950003091E40289EB90E0AC01249FC001259FE7
:10396000900D349F900D112464E670E00E94F439AC
:103970004B01AA24BB24C501B4012AE030E040E099
:1039800050E00E941B3A69017A0100E320E043E025
:103990006AE0CE010E943C073E01680E711C8EE277
:1039A000E3018993C501B4012AE030E040E050E032
:1039B0000E941B3A6B017C0100E020E041E06AE0DC
:1039C000CE010E943C07C80FD11DFE0111935F017B
:1039D0008BE489838AE2818342E050E0A40EB51E25
:1039E00085E392E00E9413169927AA27BB276C0152
:1039F0007D0100E320E042E060E1C5010E943C0758
:103A0000A80EB11CF5018DE081938AE0E501898360
:103A1000118264E372E0C2010E94470280910703B1
:103A20008E7F809307038091E5028E7F8093E5026D
:103A3000DF91CF911F910F91FF90EF90DF90CF908A
:103A4000BF90AF909F908F907F906F905F904F90BE
:103A500008952F923F924F925F926F927F928F9232
:103A60009F92AF92BF92CF92DF92EF92FF920F930D
:103A70001F93CF93DF93CDB7DEB722970FB6F8949D
:103A8000DEBF0FBECDBF9A8389836EE170E00E94D6
:103A90006A02882309F4C7C06091ED027091EE02BA
:103AA0008827992721E331E040E050E00E94C9399E
:103AB0002AE030E040E050E00E941B3A39014A0120
:103AC00066ED72E084E392E00E946B3962E771E098
:103AD00087E392E00E945639C401B30128EE33E037
:103AE00040E050E00E941B3A19012A0169017A0165
:103AF00000E320E043E06AE08BE392E00E943C07B1
:103B0000A82EBB248BE392E0A80EB91E1EE2D501BD
:103B10001D935D016218730884089508C401B30100
:103B20002AE030E040E050E00E941B3A69017A014F
:103B300000E020E042E06AE0C5010E943C07F50198
:103B4000E80FF11D8CE2DF018D935D018091F002A1
:103B50009091F10297FF05C08DE281830894A11C2A
:103B6000B11C8091F0029091F10268EE73E00E9426
:103B7000083A882777FD8095982F6B017C0100E338
:103B80002DE242E06AE0C5010E943C07F501E80F22
:103B9000F11D11935F018091F0029091F10268EEA6
:103BA00073E00E94083A6C01EE24D7FCE094FE2CEE
:103BB000F7FE08C0F094E094D094C094C11CD11CCE
:103BC000E11CF11C00E320E043E06AE0C5010E9433
:103BD0003C07A80EB11C8AE2F50181935F0185E3E1
:103BE00092E00E9413169927AA27BB276C017D013A
:103BF00020E042E060E1C5010E943C07A80EB11C34
:103C0000D5018DE08D938AE0F5018183FD0111825C
:103C100064E372E089819A810E9447028091F202F6
:103C20008E7F8093F20222960FB6F894DEBF0FBE0D
:103C3000CDBFDF91CF911F910F91FF90EF90DF905B
:103C4000CF90BF90AF909F908F907F906F905F903C
:103C50004F903F902F9008953F924F925F926F92B6
:103C60007F928F929F92AF92BF92CF92DF92EF920C
:103C7000FF920F931F93CF93DF93CDB7DEB72297B9
:103C80000FB6F894DEBF0FBECDBF9A8389836EE175
:103C900070E00E946A02882309F4C3C08091ED029B
:103CA0009091EE022C01440C551C480E591E6624BE
:103CB000772466ED72E084E392E00E946B3967E757
:103CC00071E087E392E00E9456398091ED02909175
:103CD000EE026AE070E00E94F439882799276B01B0
:103CE0007C0100E320E043E06AE08BE392E00E9485
:103CF0003C07882E99248BE392E0880E991E7EE281
:103D0000372EF40131924F018091ED029091EE0235
:103D10006AE070E00E94F439AA27BB276C017D019C
:103D200000E020E042E06AE0CF010E943C07880EFC
:103D3000911C1CE2F40111935F0186E6F40181837A
:103D4000F501118382E090E0A80EB91EC301B20113
:103D500024E630E040E050E00E941B3A69017A011D
:103D600000E320E043E06AE0C5010E943C07A80EA2
:103D7000B11CF50131925F01C301B20124E630E0CC
:103D800040E050E00E941B3A6B017C0100E020E023
:103D900043E06AE0C5010E943C07A80EB11CF50192
:103DA00011939F018DE4F5018183D9011196F901E9
:103DB00011839D012F5F3F4FFD011183590108942D
:103DC000A11CB11C86E4F90181838AE2F50181839B
:103DD00082E090E0A80EB91E85E392E00E941316DF
:103DE0009927AA27BB276C017D0100E320E042E070
:103DF00060E1C5010E943C07A80EB11CD5018DE011
:103E00008D938AE0F5018183FD01118264E372E004
:103E100089819A810E9447028091F2028E7F80936D
:103E2000F20222960FB6F894DEBF0FBECDBFDF912F
:103E3000CF911F910F91FF90EF90DF90CF90BF90A7
:103E4000AF909F908F907F906F905F904F903F903A
:103E500008958F929F92AF92BF92CF92DF92EF928E
:103E6000FF920F931F93CF93DF934C016EE170E0AD
:103E70000E946A02882309F4A4C066ED72E084E31C
:103E800092E00E946B396CE771E087E392E00E9458
:103E90005639C0902D03D0902E03D694C794EE24AB
:103EA000FF2400E320E043E06AE08BE392E00E941D
:103EB0003C07A82FBB27A55CBD4F80912D03909197
:103EC0002E0380FF08C0FD018EE2819385E3ED01A2
:103ED0008983DF0111961CE2FD0111935F0182E5E8
:103EE000ED0189831183E2E0F0E0AE0EBF1E809108
:103EF0003203909133036AE070E00E94F43988271E
:103F000099276B017C0100E320E043E06AE0C501F2
:103F10000E943C07A80EB11C8EE2E50189935E0168
:103F200080913203909133036AE070E00E94F4398B
:103F3000AA27BB276C017D0120E041E06AE0CE01A9
:103F40000E943C07A80EB11CF50111938EE4E50117
:103F50008983DF01119611835D010894A11CB11CB6
:103F600081E4FD0181838AE2E5018983E2E0F0E0FA
:103F7000AE0EBF1E85E392E00E9413169927AA2772
:103F8000BB276C017D0120E042E060E1C5010E9499
:103F90003C07A80EB11CF5018DE081938AE0E50194
:103FA0008983118264E372E0C4010E944702809118
:103FB0002F038E7F80932F03809134038E7F809315
:103FC0003403DF91CF911F910F91FF90EF90DF901D
:103FD000CF90BF90AF909F908F9008958F929F92B7
:103FE000AF92BF92CF92DF92EF92FF920F931F9307
:103FF000CF93DF93EC010E94723901C0E9018991EE
:104000009E018C32D9F7CE010E940639082F01C0DB
:10401000219688818C3239F0882359F08D3049F00F
:104020008A30B1F706C0CE010196073109F0A4C06D
:104030008FC0073149F4A7E1B0E00E94B039F09396
:10404000CA01E093C9010CC0A02FBB27A050B0400B
:104050000E94A339802D99279093CA018093C901AA
:104060000E9480054C0164E170E00E946A0288238E
:1040700009F48BC061E871E084E392E00E94563954
:10408000C02EDD24EE24FF2400E220E042E06AE0BE
:104090008BE392E00E943C07E82FFF27E55CFD4F91
:1040A000EF018CE289932091C9013091CA0137FF59
:1040B0000BC08DE28183219688279927821B930B61
:1040C0009093CA018093C9018091C9019091CA015E
:1040D00068EE73E00E94083A882777FD8095982F54
:1040E0006B017C0100E220E042E06AE0CE010E9428
:1040F0003C075E01A80EB11C8EE2D5018D935D01D7
:104100008091C9019091CA0168EE73E00E94083A5B
:104110009093CA018093C901AA2797FDA095BA2F51
:104120006C017D0100E320E043E06AE0C5010E94EC
:104130003C07A80EB11CF5018DE081938AE0E501F2
:104140008983118264E372E0C4010E9447021DC0AA
:104150000E9406399093CA018093C901A7E1B0E09B
:104160000C010E94C1398091C9019091CA019093BC
:10417000F1028093F00209C01127005010400E9404
:104180000639D801082E0E94B539DF91CF911F91D1
:104190000F91FF90EF90DF90CF90BF90AF909F90E6
:1041A0008F900895EF92FF920F931F93CF93DF9319
:1041B000CDB7DEB72A970FB6F894DEBF0FBECDBFDE
:1041C0008C01FC01628173817E010894E11CF11C69
:1041D000C7010E946B391F82CE0105960E940639E5
:1041E000809351031D82CE0103960E94063980936D
:1041F00050031B82C7010E94063980934F038091B0
:104200004E03806B80934E030E94E109809352031A
:10421000F801848195810E94063980935703F80143
:10422000868197810E94063980935603F801808524
:1042300091850E940639805D8093550380915403D7
:10424000806B809354030E94E1098093580380910E
:10425000E20280698093E2022A960FB6F894DEBFEC
:104260000FBECDBFDF91CF911F910F91FF90EF90C7
:104270000895CF93DF93EC01EA81FB81808188234D
:10428000A9F0CF010E94063990931D0380931C036F
:104290008091E20280698093E20280911E03806B2C
:1042A00080931E030E94E10980931F03DF91CF9149
:1042B0000895CF92DF92EF92FF920F931F93CF93C7
:1042C000DF93CDB7DEB724970FB6F894DEBF0FBEED
:1042D000CDBF7C01FC0180818C3241F480916F0361
:1042E0008F7680936F0380E090E06CC0882311F498
:1042F00000E060C01B821C82D7018D918983F70189
:1043000081818A838D010F5F1F4FFD0181818B8326
:1043100078010894E11CF11C8091E202806980938D
:10432000E20280916F03806B80936F036E010894AB
:10433000C11CD11CC6010E94063980936E03F8018E
:104340008181898387010F5F1F4FF70181818A83F4
:1043500078010894E11CF11C1B82C6010E940639F9
:1043600080937003F80181818E3211F005E022C044
:10437000D7011196F701818189837D010894E11CA1
:10438000F11C1A82FD019181892F80538A3010F02F
:1043900007E006C09A830894E11CF11C1B8208E028
:1043A000C6010E9406398093710304C00894E11C81
:1043B000F11C0F5FF70180818C3211F08823B1F777
:1043C000802F992724960FB6F894DEBF0FBECDBF7D
:1043D000DF91CF911F910F91FF90EF90DF90CF90E1
:1043E0000895CF92DF92EF92FF920F931F93CF9396
:1043F000DF93CDB7DEB723970FB6F894DEBF0FBEBD
:10440000CDBF7C01FC0180818C3241F480916B0333
:104410008F7680936B0380E090E05FC0882309F47F
:1044200055C01B82F70181918F018983F70181813A
:104430008A8378010894E11CF11C8091E202806972
:104440008093E20280916B03806B80936B036E011B
:104450000894C11CD11CC6010E94063980936A03CE
:104460000E94E10980937403F801818189838701A7
:104470000F5F1F4FF70181818A8378010894E11C47
:10448000F11CC6010E94063980936C03F8018181FA
:104490008E32A1F4D7011196F70181818983FD0144
:1044A00081818A8312E0E12EF12CEA0EFB1EC60107
:1044B0000E94063980936D0387E008C010926D0357
:1044C00084E004C00894E11CF11C8F5FF701908127
:1044D0009C3211F09923B1F7992723960FB6F894DF
:1044E000DEBF0FBECDBFDF91CF911F910F91FF9027
:1044F000EF90DF90CF900895CF92DF92EF92FF92EE
:104500000F931F93CF93DF93CDB7DEB723970FB6EB
:10451000F894DEBF0FBECDBF6C01FC0180818C32F0
:1045200041F4809154038F768093540380E090E0AF
:1045300050C0882309F446C01B82F60181918F0187
:104540008983F60181818A8368010894C11CD11C8A
:104550008091E20280698093E20280915403806B33
:10456000809354037E010894E11CF11CC7010E9452
:10457000063980935703F8018181898386010F5F93
:104580001F4FF60181818A8368010894C11CD11CE8
:10459000C7010E94063980935603F80181818983FF
:1045A000F60181818A8382E090E0C80ED91EC7019E
:1045B0000E9406398093550386E004C00894C11C0C
:1045C000D11C8F5FF60190819C3211F09923B1F7D5
:1045D000992723960FB6F894DEBF0FBECDBFDF91AB
:1045E000CF911F910F91FF90EF90DF90CF900895A2
:1045F000CF92DF92EF92FF920F931F93CF93DF93AF
:10460000CDB7DEB724970FB6F894DEBF0FBECDBF8F
:104610007C01FC0180818C3241F48091FC028F7618
:104620008093FC0280E090E070C0882311F400E0E9
:1046300064C01B821C82D7018D918983F70181811F
:104640008A838D010F5F1F4FFD0181818B8378016C
:104650000894E11CF11C8091E20280698093E202DF
:104660008091FC02806B8093FC026E010894C11C57
:10467000D11CC6010E9406398093FB020E94E10909
:104680008093FD02F8018181898387010F5F1F4FAD
:10469000F70181818A8378010894E11CF11C1B8257
:1046A000C6010E9406398093FF02F80181818E3293
:1046B00011F005E022C0D7011196F70181818983AD
:1046C0007D010894E11CF11C1A82FD019181892F62
:1046D00080538A3010F007E006C09A830894E11CEA
:1046E000F11C1B8208E0C6010E940639809300037A
:1046F00004C00894E11CF11C0F5FF70180818C322B
:1047000011F08823B1F7802F992724960FB6F894DB
:10471000DEBF0FBECDBFDF91CF911F910F91FF90F4
:10472000EF90DF90CF900895CF92DF92EF92FF92BB
:104730000F931F93CF93DF93CDB7DEB723970FB6B9
:10474000F894DEBF0FBECDBF7C01FC0180818C32AE
:1047500041F48091F6028F768093F60280E090E03B
:104760005FC0882309F455C01B82F70181918F0136
:104770008983F70181818A8378010894E11CF11C07
:104780008091E20280698093E2028091F602806B60
:104790008093F6026E010894C11CD11CC6010E94D0
:1047A00006398093F5020E94E1098093F702F8012F
:1047B0008181898387010F5F1F4FF70181818A8380
:1047C00078010894E11CF11CC6010E94063980930F
:1047D000F902F80181818E32A1F4D7011196F70117
:1047E00081818983FD0181818A8302E0E02EF12CA1
:1047F000EA0EFB1EC6010E9406398093FA0287E08A
:1048000008C01092FA0284E004C00894E11CF11C74
:104810008F5FF70190819C3211F09923B1F79927AE
:1048200023960FB6F894DEBF0FBECDBFDF91CF91B8
:104830001F910F91FF90EF90DF90CF9008958F928E
:104840009F92AF92BF92CF92DF92EF92FF920F931F
:104850001F93CF93DF93CDB7DEB723970FB6F894AE
:10486000DEBF0FBECDBF7C01FC0180818C3241F4E4
:1048700080914E038F7680934E0380E090E081C05C
:10488000882309F477C01B82F70181916F01898326
:10489000F70181818A8356010894A11CB11C4E0145
:1048A0000894811C911C00914F031127C4010E94A0
:1048B00006390817190779F08091E2028069809320
:1048C000E20280914E03806B80934E03C4010E94EC
:1048D000063980934F03F60181818983750108941D
:1048E000E11CF11CF50181818A8367010894C11CD8
:1048F000D11C009150031127C4010E9406390817EA
:10490000190779F08091E20280698093E202809138
:104910004E03806B80934E03C4010E94063980933E
:104920005003F70181818983F60181818A8382E0C6
:10493000E82EF12CEC0CFD1C009151031127C40151
:104940000E9406390817190779F08091E202806900
:104950008093E20280914E03806B80934E03C401EA
:104960000E9406398093510386E004C00894E11C3C
:10497000F11C8F5FF70190819C3211F09923B1F700
:10498000992723960FB6F894DEBF0FBECDBFDF91F7
:10499000CF911F910F91FF90EF90DF90CF90BF903C
:1049A000AF909F908F9008950F931F93CF93DF93B5
:1049B000FC0101C0FE018191EF018C32D9F7CF01DA
:1049C0000E949423FE01E80FF11D80818C3209F0D2
:1049D0003FC09F012F5F3F4F81818E3411F083359F
:1049E00021F4809301032F5F3F4F89010F5F1F4F19
:1049F000C8010E94F822F801E80FF11D80818C3275
:104A000039F59F012F5F3F4F0181053411F00735C4
:104A100021F4009302032F5F3F4F89010F5F1F4F67
:104A2000C8010E941F24F801E80FF11D80818C321B
:104A300079F48091E20280698093E2028181909111
:104A40000303813411F0906101C09F7E90930303B2
:104A5000DF91CF911F910F910895DF92EF92FF9216
:104A60000F931F93CF93DF937C01EB01D42E042F80
:104A70001127CB010E940639089F9001099F300D34
:104A8000189F300D1124D7012D933C93FE0101C0D6
:104A900031966E2F6C1B4081842F9927C0970A97FF
:104AA000B8F34E32B9F5DF0111967181472F5527C2
:104AB000CA01C0970A9770F56F5FEAE0DE1621F031
:104AC000F4E6DF1651F007C020533040240F351FA5
:104AD000E70139832883FD011DC0205E31408AE053
:104AE000789FC0011124280F391FF70131832083DB
:104AF000FD0131966F5FED0189819927C0978A305A
:104B0000910540F4820F931FD7018D939C9302C0AF
:104B10006F5F319680818C3221F0882311F08A32C8
:104B2000B9F7862F9927DF91CF911F910F91FF90B1
:104B3000EF90DF9008950F931F93CF93DF93CDB73E
:104B4000DEB722970FB6F894DEBF0FBECDBFFC01D3
:104B500001C0F80181918F018C32D9F741E0BF018A
:104B6000CE0101960E942D25F801E80FF11D8081EC
:104B70008C32B9F481818D34A1F489819A8190932A
:104B80001D0380931C038091E20280698093E202FE
:104B900080911E03806B80931E030E94E109809325
:104BA0001F0322960FB6F894DEBF0FBECDBFDF9174
:104BB000CF911F910F910895EF92FF920F931F9342
:104BC000CF93DF93CDB7DEB722970FB6F894DEBF51
:104BD0000FBECDBFFC0101C0F80181918F018C3265
:104BE000D9F74AE0BF017E010894E11CF11CC7011E
:104BF0000E942D25F801E80FF11D80818C3209F00B
:104C000047C0DF01119681818C3209F011968C9199
:104C10008C32F1F58D010F5F1F4F4AE0B801C701DB
:104C20000E942D25F801E80FF11D80818C3281F55D
:104C3000DF01119681818C3209F011968C918C32B2
:104C400039F58D010F5F1F4F4AE0B801C7010E947F
:104C50002D25F801E80FF11D80818C32C9F4018106
:104C60000C32B1F00E34A1F489819A819093E40260
:104C70008093E3028091E20280698093E202809156
:104C8000E502806B8093E5020E94E1098093E602D1
:104C900022960FB6F894DEBF0FBECDBFDF91CF9145
:104CA0001F910F91FF90EF900895FC016281738135
:104CB0004AE08FEC91E00E942D256091CF01709128
:104CC000D0018827992728E431E040E050E00E9495
:104CD000C9396093CB017093CC018093CD0190933F
:104CE000CE0124E630E040E050E00E941B3A3093D1
:104CF000EE022093ED028091E20280698093E2024D
:104D00008091F202806B8093F2020E94E10980930D
:104D1000F3020895EF92FF920F931F93CF93DF93C7
:104D2000CDB7DEB722970FB6F894DEBF0FBECDBF6A
:104D3000FC01A89B02C0A89803C0A89A01C03196A4
:104D400080818C32E1F72CC08F010F5F1F4F4AE04A
:104D5000B801C7010E942D25F801E80FF11D8081DF
:104D60008C3229F59F012F5F3F4F81818636A9F450
:104D700089819A819093EE028093ED028091E20204
:104D800080698093E2028091F202806B8093F2024C
:104D90000E94E1098093F3020AC0F901319604C030
:104DA0007E010894E11CF11C80818C3269F222960C
:104DB0000FB6F894DEBF0FBECDBFDF91CF911F912C
:104DC0000F91FF90EF900895CF93DF93FC0101C006
:104DD000FE018191EF018C32D9F74AE0BF0186E2F2
:104DE00093E00E942D25FE01E80FF11D80818C3299
:104DF00011F0833489F48181833471F48091E2026B
:104E000080698093E20280912803806B809328035D
:104E10000E94E10980932903DF91CF910895CF93F8
:104E2000DF93EC018881909118038C3231F49F76E6
:104E30009093180380E090E013C08091E2028069B3
:104E40008093E202906B909318030E94E109809393
:104E500019034AE0BE0186E193E00E942D259927BF
:104E6000DF91CF910895CF93DF93EC0188819091EA
:104E70000C038C3231F49F7690930C0380E090E029
:104E800013C08091E20280698093E202906B90935C
:104E90000C030E94E10980930D0344E6BE018AE001
:104EA00093E00E942D259927DF91CF9108951F93BC
:104EB000CF93DF93EC018881909107038C3231F41A
:104EC0009F769093070380E090E033C08091E202E8
:104ED00080698093E202906B909307030E94E1093E
:104EE000809308034AE0BE0185E093E00E942D25EF
:104EF000182F8091D5028823D1F0809105039091DD
:104F000006036AE070E00E94F43970931D03609319
:104F10001C038091E20280698093E20280911E036B
:104F2000806B80931E030E94E10980931F03812FF1
:104F30009927DF91CF911F9108951F93CF93DF930E
:104F4000EC0188819091EA028C3231F49F76909343
:104F5000EA0280E090E031C08091E20280698093B3
:104F6000E202906B9093EA020E94E1098093EB02C7
:104F70004AE0BE0188EE92E00E942D25182FAEE097
:104F8000B0E00E94A339802D8823A9F48091E50226
:104F90008C688093E5020E94E1098093E6020E94FA
:104FA000E1098093E7028091E8029091E9029093F1
:104FB000E4028093E302812F9927DF91CF911F9123
:104FC0000895CF93DF93FC0101C0FE018191EF01B1
:104FD0008C32D9F7CF010E945727FE01E80FF11D4F
:104FE00080818C3269F4319680818D3429F08A3247
:104FF00039F08823C1F704C0CF0102960E949D2793
:10500000DF91CF9108950F931F93CF93DF93FC010E
:1050100001C0FE018191EF018C32D9F7CF010E94CE
:105020001F24FE01E80FF11D80818C3209F05FC062
:105030008091E20280698093E202AF014F5F5F4F8F
:10504000818120910303813411F0206101C02F7E02
:10505000209303038A010E5F1F4FC8010E9494230F
:10506000F801E80FF11D80818C3209F040C09F01EA
:105070002F5F3F4F01810E3411F0033521F400936F
:1050800001032F5F3F4F89010F5F1F4FC8010E942F
:10509000F822F801E80FF11D80818C3241F59F0163
:1050A0002F5F3F4F0181053411F0073521F4009344
:1050B00002032F5F3F4F89010F5F1F4FC8010E94FE
:1050C0009D27F801E80FF11D80818C3281F48F015A
:1050D0000F5F1F4FC8010E945727F801E80FF11D0D
:1050E00080818C3221F4CF0101960E947C22DF91D5
:1050F000CF911F910F910895CF92DF92EF92FF927F
:105100000F931F93CF93DF93CDB7DEB7A6970FB65C
:10511000F894DEBF0FBECDBF8C011A8219820E94A7
:10512000723902C00F5F1F4FF80180818C32D1F7B6
:105130007E010894E11CF11CCC24CA94DD2420C01B
:105140000F5F1F4FC8010E9427169927F70191830F
:105150008083D394CC2021F080509F4F9183808313
:1051600082E090E0E80EF91E02C00F5F1F4FF801C9
:105170008081CC248C3221F0882311F08A32A9F767
:10518000F80180818823E1F66D2DCE0101960E9401
:105190005C10A6960FB6F894DEBF0FBECDBFDF91B0
:1051A000CF911F910F91FF90EF90DF90CF900895D6
:1051B000BF92CF92DF92EF92FF920F931F93CF9304
:1051C000DF936C01EB01B42EE42EFF24002711279E
:1051D000CB010E9424399B01AC01C801B7010E9498
:1051E000C9397B018C01D6016D937D938D939C937E
:1051F0001397FE0101C031966E2F6C1B2081822F08
:105200009927C0970A97B8F32E3209F050C0EF01E2
:1052100021962181822F9927C0978A30910508F025
:1052200046C06F5FBAE0BB1621F0E4E6BE1681F01F
:105230000DC0AA2797FDA095BA2F8E0D9F1DA01F08
:10524000B11FF60180839183A283B383FE012FC037
:105250008AE0289FC0011124805E91409C01442770
:1052600037FD4095542F2E0D3F1D401F511FD60175
:105270002D933D934D935C931397FE0131966F5F91
:1052800089819927C0978A30910588F4AA2797FDCC
:10529000A095BA2F280F391F4A1F5B1FD6012D93E7
:1052A0003D934D935C93139702C06F5F319680815D
:1052B0008C3221F0882311F08A32B9F7862F992792
:1052C000DF91CF911F910F91FF90EF90DF90CF90E2
:1052D000BF900895EF92FF920F931F93CF93DF93A8
:1052E000CDB7DEB724970FB6F894DEBF0FBECDBFA3
:1052F000FC0101C0F80181918F018C32D9F74AE09D
:10530000BF017E010894E11CF11CC7010E94D8284E
:10531000F801E80FF11D80818C3209F06DC08F011A
:105320000F5F1F4F8181823509F066C069817A81E4
:105330008B819C8125E030E040E050E00E941B3AE8
:1053400030932E0320932D038091E2028069809395
:10535000E20280912F03806B80932F030E94E1096A
:10536000809330030E5F1F4F4AE0B801C7010E94CF
:10537000D828080F111DF80180818C32E9F5818150
:105380008E34A1F489819A81909333038093320300
:105390008091E20280698093E20280913403806B05
:1053A000809334030E94E10980933503F8018181E1
:1053B0008B3411F569817A818B819C8124E630E000
:1053C00040E050E00E94C93929EB30E040E050E075
:1053D0000E941B3A30933303209332038091E20200
:1053E00080698093E20280913403806B8093340360
:1053F0000E94E1098093350324960FB6F894DEBF2E
:105400000FBECDBFDF91CF911F910F91FF90EF9015
:105410000895EF92FF920F931F93CF93DF93CDB731
:10542000DEB724970FB6F894DEBF0FBECDBFFC01E8
:1054300001C0F80181918F018C32D9F74AE0BF0198
:105440007E010894E11CF11CC7010E94D828F801D4
:10545000E80FF11D80818C3209F04DC09F012F5F54
:105460003F4F81818E34B1F489819A81AB81BC81B7
:1054700080933C0390933D03A0933E03B0933F037E
:105480008091E20280698093E20280914003806B08
:105490008093400389010F5F1F4FF90181818C3296
:1054A00051F50F5F1F4F44E6B801C7010E94D8288D
:1054B000F801E80FF11D80818C32E9F481818E348E
:1054C000D1F489819A81AB81BC8180933703909319
:1054D0003803A0933903B0933A038091E2028069C4
:1054E0008093E20280913B03806B80933B030E9498
:1054F000E1098093410324960FB6F894DEBF0FBEF6
:10550000CDBFDF91CF911F910F91FF90EF90089544
:10551000CF93DF93EC018881909113038C3231F4A7
:105520009F769093130380E090E013C08091E20295
:1055300080698093E202906B909313030E94E109CB
:105540008093140344E6BE018FE093E00E94D828C4
:105550009927DF91CF9108950F931F93FC0101C00C
:10556000FD01DF018D918C32D9F7818120910303F8
:10557000813411F0206101C02F7E209303038D013F
:105580000E5F1F4FC8010E943327F801E80FF11D7D
:1055900080818C3209F09CC0DF01119680E28093FB
:1055A00004038181823511F48093040301810C345A
:1055B00011F4009304039D012F5F3F4FFD01818192
:1055C0008C3209F085C089010F5F1F4F45E06EE501
:1055D00073E0C8010E94B715F801E80FF11D808142
:1055E0008C3209F075C08F010F5F1F4F45E064E6F4
:1055F00073E0C8010E94B71590917603882311F0DB
:10560000906B01C09F7690937603F801E80FF11D2F
:1056100080818C3209F05CC08F010F5F1F4FC80181
:105620000E94F121F801E80FF11D80818C3209F010
:105630004FC09F012F5F3F4F81818E3411F0833522
:1056400051F58093720389010E5F1F4FC8010E94BC
:105650005921F801E80FF11D80818C32C9F59F01B5
:105660002F5F3F4F8181853411F08735A1F48093FE
:10567000730389010E5F1F4F8091E202806980935E
:10568000E202C8010E94882AF801E80FF11D80811A
:105690008C32F1F406C0809176038F768093760386
:1056A00017C08F010F5F1F4FC8010E940F27F8011D
:1056B000E80FF11D80818C3259F48FEF80931B032A
:1056C00081818C3229F08D3019F031968823C1F711
:1056D0001F910F9108950F931F93CF93DF93EC01C8
:1056E0008C010E5F1F4F43E050E065EC71E0C80194
:1056F0000E945D39892B21F4CE010E94AC2AC4C0DE
:1057000043E050E061EC71E0C8010E945D39892BF3
:1057100021F4CE010E940328B7C043E050E06DEBB6
:1057200071E0C8010E945D39892B21F4CE010E94ED
:10573000D424AAC043E050E069EB71E0C8010E94A4
:105740005D39892B21F4CE010E94E1279DC043E001
:1057500050E065EB71E0C8010E945D39892B21F4AE
:10576000CE010E94E42690C043E050E061EB71E07E
:10577000C8010E945D39892B21F4CE010E948A263E
:1057800083C043E050E06DEA71E0C8010E945D39DA
:10579000892B21F4CE010E94092A76C043E050E013
:1057A00069EA71E0C8010E945D39892B21F4CE01BC
:1057B0000E946A2969C043E050E065EA71E0C801CF
:1057C0000E945D39892B21F4CE010E94DC255CC04A
:1057D00043E050E061EA71E0C8010E945D39892B25
:1057E00021F4CE010E949B254FC045E050E06BE9BB
:1057F00071E0CE010E945D39892B21F4CE010E9417
:105800007C2842C045E050E065E971E0CE010E948D
:105810005D39892B21F4CE010E94EE1F35C044E191
:1058200050E068ED71E0CE010E94E015C091D80112
:10583000D091D901229643E050E061E971E0CE01B8
:105840000E945D39892B29F488ED91E00E9455264C
:105850001BC043E050E06DE871E0CE010E945D396D
:10586000892B29F488ED91E00E9439210DC043E095
:1058700050E069E871E0CE010E945D39892B21F486
:1058800088ED91E00E94D220DF91CF911F910F917E
:1058900008951F93282F843271F48FEF809378033B
:1058A00081E090E09093D7018093D6011092D501CA
:1058B0001092D101BCC08D3011F08A3031F483E0F8
:1058C00090E09093D7018093D6018091D60190917A
:1058D000D7018130910569F08130910538F082302F
:1058E000910579F1039709F0A2C051C01092780395
:1058F0009EC02A3239F482E090E09093D7018093E1
:10590000D60193C08091D10182278093D1018091EB
:10591000D501E82FFF27E958FC4F2283182F1F5F7E
:105920001093D501E12FFF27E958FC4F1282822FF7
:1059300099270E949B39892B09F1103508F477C00B
:105940001DC08091D501882331F42093D20181E0DC
:105950008093D5016CC083E090E09093D701809351
:10596000D6012093D3011092D40182ED91E00E94E0
:1059700027169091D101891709F459C01092D701C7
:105980001092D6011092D5011092790350C08091E7
:10599000D501882309F443C0A4E0B0E00E94A339F4
:1059A000802D882331F480917903883511F0883770
:1059B00079F58FEF8093C8010E94800564E20E9410
:1059C00022020E94800569E773E00E9447028091ED
:1059D000D201882329F00E9480056AE20E942202F7
:1059E0000E94800562ED71E00E9447020E948005DE
:1059F0006DE00E9422020E9480056AE00E9422025D
:105A00000E9462061092C8011092D2011092D30136
:105A100089E793E00E946B2B8FEF809377031092BE
:105A2000D7011092D601109278031092D5011F91E0
:105A30000895CF93DF930E948005EC018091FC02D2
:105A4000282F332720FF17C08091F60280FF13C054
:105A500025FD11C08091E102882319F0CE010E943A
:105A600070180E9462068091070380FFA3C0CE01D8
:105A70000E94C6169FC08091E502282F3327C901D6
:105A800089709070892B69F0A6E0B0E00E94A3397C
:105A9000802D882331F025FD04C0CE010E94D91B42
:105AA00089C080911E03282F332720FF0DC0A7E057
:105AB000B0E00E94A339802D882331F025FD04C079
:105AC000CE010E946D1B76C080912F0380FF12C013
:105AD000A8E0B0E00E94A339802D882359F080917E
:105AE0003403992780FF06C085FD04C0CE010E94C3
:105AF000291F60C08091F202282F332720FF18C091
:105B0000A9E0B0E00E94A339802D882389F025FD0B
:105B10000FC08091F0029091F1028F5F9F4F21F4AE
:105B2000CE010E942C1E46C0CE010E94291D42C0FB
:105B300080912803282F332720FF0DC0AAE0B0E072
:105B40000E94A339802D882331F025FD04C0CE01A9
:105B50000E947B192FC080913B03282F332720FD03
:105B600004C08091400380FF0DC0ABE0B0E00E9414
:105B7000A339802D882331F025FD04C0CE010E9479
:105B80000D1A18C080914B03282F332720FF0DC01A
:105B9000AAE1B0E00E94A339802D882331F025FDD1
:105BA00004C0CE010E94EB1A05C08091E2028E7FF4
:105BB0008093E202DF91CF910895CF93DF93ADE020
:105BC000B0E00E94A339802D882341F164E271E0A6
:105BD00084E392E00E94563969E171E04A960E949E
:105BE0005639EC016AE071E00A960E945639FE01CE
:105BF0007896AEE0B0E00E94A339802D882339F476
:105C000060E071E0CF010E945639FE01B19610822A
:105C10000E94800564E372E00E944702DF91CF9109
:105C200008958091E50280688093E5028091EA0200
:105C300080688093EA028091F20280688093F20289
:105C40008091F60280688093F6028091FC02806861
:105C50008093FC0280910703806880930703809102
:105C60000C03806880930C038091130380688093F9
:105C700013038091180380688093180380911E039A
:105C8000806880931E0380912303806880932303A0
:105C90008091280380688093280380912C0380687A
:105CA00080932C0380912F03806880932F03809131
:105CB000340380688093340380913B038068809331
:105CC0003B038091400380688093400380914403AC
:105CD00080688093440380914703806880934703E2
:105CE00080914B03806880934B0380914E038068C2
:105CF00080934E0380915403806880935403809175
:105D00005B03806880935B03809176038068809357
:105D1000760308959E9B02C09F991AC080916200ED
:105D2000882331F00E94E109809301021092620001
:105D3000809162008823F9F4809101020E94E509B4
:105D40008430C8F08FEF8093620082E090E0089585
:105D500080916200882379F48FEF809362008091B4
:105D600001020E94E50920E030E0882311F021E0E3
:105D700030E0C901089580E090E00895CCE5D8E0D6
:105D8000DEBFCDBF40E250E06CE872E087E892E011
:105D90000E9482020E94CC090E94000A0E943805DB
:105DA0000E946C0484E28093D60282E027ED32E008
:105DB000A2E0B0E0F901182E0E94AB398091D70221
:105DC0008F3F29F469E373E0C9010E9456391092AC
:105DD000D9020E944906AFE0B0E00E94A339802DAD
:105DE0008093DA02A0E1B0E00E94A339802D809375
:105DF000DB02A1E1B0E00E94A339802D80938602EE
:105E0000A2E1B0E00E94A339802D8093D402A3E1E7
:105E1000B0E00E94A339802D8093E002A6E1B0E0BB
:105E20000E94A339802D8093E102ACE1B0E00E9492
:105E3000A339802D882319F01092D50203C081E088
:105E40008093D502A4E1B0E00E94A339802D809315
:105E5000EF02A7E1B0E00E94B039F093F102E093C5
:105E6000F002A1E0B0E00E94A339802D853039F125
:105E7000863028F4833051F0843009F50CC0873027
:105E8000A1F0873068F08830D1F414C060EB74E082
:105E900080E090E018C060E679E080E090E013C018
:105EA00060E875E280E090E00EC060E07BE480E0B6
:105EB00090E009C060E076E980E090E004C060EC2A
:105EC00072E180E090E00E9463050E94C60880E5D0
:105ED0000E94D1080E94990A84EF91E00E94410833
:105EE000A09A0E94750A82E49AE00E947C0685E2EC
:105EF00093E00E94620A61E080E00E94860A82E1EB
:105F000093E00E94620A62E080E00E94860A82E0DA
:105F100093E00E94620A63E080E00E94860A87EFB5
:105F200092E00E94620A8CED95E00E9441080E9476
:105F3000112E8091E20280688093E2021092790330
:105F40001092780387B3896087BBC39AC09A84B3E1
:105F50008F7384BB85B3806C85BB8F9A979A84B30B
:105F60008F6084BB85B38F6085BB0E94E109982E4A
:105F70000E94DD2D0E94620688E190E02EE00FB6BF
:105F8000F894A89581BD0FBE21BD3E010894611C07
:105F9000711C62E0462E512C4C0E5D1E57E8C52E3A
:105FA00052E0D52E47E2242E42E0342E39ECA32EC7
:105FB00031E0B32E8091E20280FF04C00E94192DCF
:105FC0000E9462060E94EC10C3010E941C068823F6
:105FD00019F089810E94492CC2010E94F50488238E
:105FE00021F08A819B810E94C70AC6010E94210379
:105FF0008823D9F160910002662339F0C6010E941E
:10600000C6028F3F910509F038F410910002C601D5
:106010000E942103181790F01092000207C0C601D9
:106020000E94B1028F3F910509F040F4C6010E9421
:106030008902C6010E942103882389F70E9468040F
:10604000882329F00E946C04109200020EC0609117
:106050000002C6010E94C6020E944C03882329F058
:10606000809100028F5F80930002A8958091E202E8
:1060700087FD33C20E94E109981611F40C94D238BE
:106080000E94E109982E8091EB020E94E5098F3170
:1060900068F09091EA0295FF09C09F7D8091E2022D
:1060A00080688093E20290689093EA0280910803EE
:1060B0000E94E5098F3168F09091070395FF09C0B0
:1060C0009F7D8091E20280688093E20290689093C5
:1060D00007038091E6020E94E5098F3168F09091F4
:1060E000E50295FF09C09F7D8091E2028068809360
:1060F000E20290689093E502809124030E94E509F2
:106100008F3168F09091230395FF09C09F7D8091A6
:10611000E20280688093E20290689093230380916A
:106120001F030E94E5098F3168F090911E0395FFCF
:1061300009C09F7D8091E20280688093E2029068AE
:1061400090931E038091F3020E94E5098F3168F05D
:106150009091F20295FF09C09F7D8091E2028068D4
:106160008093E20290689093F2028091F7020E947D
:10617000E5098F3168F09091F60295FF09C09F7D87
:106180008091E20280688093E20290689093F60228
:106190008091FD020E94E5098F3168F09091FC0228
:1061A00095FF09C09F7D8091E20280688093E202A2
:1061B00090689093FC02809129030E94E5098F3139
:1061C00068F09091280395FF09C09F7D8091E202BD
:1061D00080688093E2029068909328038091140372
:1061E0000E94E5098F3168F09091130395FF09C073
:1061F0009F7D8091E20280688093E2029068909394
:106200001303809119030E94E5098F3168F0909182
:10621000180395FF09C09F7D8091E20280688093FA
:10622000E20290689093180380910D030E94E509A3
:106230008F3168F090910C0395FF09C09F7D80918C
:10624000E20280688093E202906890930C03809150
:1062500058030E94E5098F3168F09091540395FF2F
:1062600009C09F7D8091E20280688093E20290687D
:1062700090935403809152030E94E5098F3168F096
:1062800090914E0395FF09C09F7D8091E202806846
:106290008093E202906890934E03809174030E9471
:1062A000E5098F3168F09091760395FF09C09F7DD5
:1062B0008091E20280688093E20290689093760376
:1062C000809135030E94E5098F3168F09091340385
:1062D00095FF09C09F7D8091E20280688093E20271
:1062E000906890933403809130030E94E5098F31C8
:1062F00068F090912F0395FF09C09F7D8091E20285
:1063000080688093E202906890932F038091EC0262
:106310000E94E5098F3168F09091EA0296FF09C06A
:106320009F7B8091E20280688093E2029068909364
:10633000EA02809109030E94E5098F3168F090918B
:10634000070396FF09C09F7B8091E20280688093DB
:10635000E2029068909307038091E7020E94E509AA
:106360008F3170F09091E502892F847449F09B7B06
:106370008091E20280688093E20290689093E50247
:10638000809125030E94E5098F3168F090912303E5
:1063900096FF09C09F7B8091E20280688093E202B1
:1063A0009068909323038091F4020E94E5098F3155
:1063B00068F09091F20296FF09C09F7B8091E20203
:1063C00080688093E20290689093F2028091F802D4
:1063D0000E94E5098F3168F09091F60296FF09C09E
:1063E0009F7B8091E20280688093E20290689093A4
:1063F000F6028091FE020E94E5098F3168F09091CB
:10640000FC0296FF09C09F7B8091E2028068809326
:10641000E20290689093FC0280912A030E94E509B1
:106420008F3168F09091280396FF09C09F7B80917F
:10643000E20280688093E202906890932803809142
:1064400053030E94E5098F3168F090914E0396FF47
:1064500009C09F7B8091E20280688093E20290688D
:1064600090934E03809159030E94E5098F3168F0A3
:106470009091540396FF09C09F7B8091E20280684F
:106480008093E202906890935403809136030E94B7
:10649000E5098F3168F09091340396FF09C09F7B26
:1064A0008091E20280688093E202906890933403C6
:1064B000809131030E94E5098F3108F473C69091F1
:1064C0002F0396FF6FC69F7B8091E20280688093C6
:1064D000E202906890932F0365C69091020291307A
:1064E00009F4ACC2913020F0923009F05BC692C43E
:1064F0008F778093E2029091E50297FF31C0892F58
:10650000847671F19F779093E50260E080E00E94CD
:10651000860A82EF92E00E94620A8091E3029091E3
:10652000E4026AE070E00E94F439882799277B0131
:106530008C0120E340E063E08AE00E9487068EE25F
:106540000E94420A8091E3029091E4026AE070E0C6
:106550000E94F439AA27BB277C018D0120E3CEC01D
:10656000892F847661F497FF0AC09F779093E502A4
:1065700060E00E94860A87EE92E00E94620A909193
:10658000EA0297FF35C0892F807691F19F7790932B
:10659000EA0260E08AE00E94860A80EE92E00E94B1
:1065A000620A8091E8029091E9026AE070E00E943C
:1065B000F439882799277B018C0120E340E062E0D1
:1065C0008AE00E9487068EE20E94420A8091E802D9
:1065D0009091E9026AE070E00E94F439AA27BB2793
:1065E0007C018D0120E340E061E08AE00E948706A3
:1065F0009091EA02892F807669F497FF0BC09F770C
:106600009093EA0260E08AE00E94860A85ED92E0BB
:106610000E94620A9091F20297FF77C0892F8076DC
:1066200009F473C09F779093F20261E080E00E94CA
:10663000860A80ED92E00E94620A6091ED027091FC
:10664000EE028827992721E331E040E050E00E94E4
:10665000C93920E137E240E050E00E941B3A79015D
:106660008A0120E340E063E08AE00E9487068EE230
:106670000E94420A6091ED027091EE0288279927EC
:1066800021E331E040E050E00E94C9397B018C01F8
:1066900020E137E240E050E00E941B3A2093DC0208
:1066A0003093DD024093DE025093DF02E092D0028D
:1066B000F092D1020093D2021093D302CA01B90121
:1066C00020E137E240E050E00E94C939E61AF70ABB
:1066D000C70164E670E00E94F4397093850260930C
:1066E00084026A30710568F480E30E94420AE090F7
:1066F0008402F09085020027112720E240E061E04B
:106700004EC57B010027112747C5892F807661F48C
:1067100097FF0AC09F779093F20261E00E94860A79
:1067200085EC92E00E94620A9091F60297FF71C098
:10673000892F807609F46DC09F779093F60262E00E
:1067400080E00E94860A80910303882329F082EC6E
:1067500092E00E94620A07C0809101030E94420AEF
:1067600080E20E94420AE090F502FF2400271127F0
:1067700020E340E062E08AE00E9487068DE20E940A
:10678000420AE090F902FF240027112720E340E0AD
:1067900062E08AE00E9487068EE20E94420AE09050
:1067A000FA02FF240027112720E340E062E08AE09C
:1067B0000E94870663E080E00E94860A80910203BF
:1067C0000E94420AE090FB02FF240027112720E3E9
:1067D00040E063E08AE00E9487068DE20E94420A60
:1067E000E090FF02FF240027112720E340E062E051
:1067F0008AE00E9487068EE20E94420AE09000032F
:10680000FF240027112720E340E062E08AE00E9495
:1068100087069091F602892F807659F497FF09C078
:106820009F779093F60262E00E94860AC5010E945B
:10683000620A9091FC02892F807659F497FF09C073
:106840009F779093FC0263E00E94860AC5010E9434
:10685000620A9091070397FF35C0892F807691F1E6
:106860009F779093070361E08AE00E94860A8CEB91
:1068700092E00E94620A80910503909106036AE00B
:1068800070E00E94F439882799277B018C0120E26F
:1068900040E063E08AE00E9487068EE20E94420A9E
:1068A00080910503909106036AE070E00E94F4393C
:1068B000AA27BB277C018D0120E340E061E08AE04C
:1068C0000E94870690910703892F807669F497FFCD
:1068D0000BC09F779093070361E08BE00E94860ACC
:1068E00082EB92E00E94620A9091340397FF54C0B9
:1068F000892F807609F450C09F779093340362E02B
:106900008AE00E94860A8BEA92E00E94620A8091E5
:10691000860220913203309133038823C9F0C901E4
:1069200064E170E00E94F439882799277B018C018B
:1069300020E340E062E08AE00E9487068EE20E9447
:10694000420A80913203909133039695879516C041
:10695000C9016AE070E00E94F439882799277B0119
:106960008C0120E340E062E08AE00E9487068EE22C
:106970000E94420A80913203909133036AE070E0F2
:106980000E94F439AA27BB277C018D0120E340E057
:1069900061E08AE00E94870690913403892F807617
:1069A00069F497FF0BC09F779093340362E08AE00D
:1069B0000E94860A80EA92E00E94620A90912F0368
:1069C00097FF2AC0892F807639F19F7790932F0304
:1069D00063E08AE00E94860A8AE992E00E94620AE5
:1069E000E0902D03F0902E03F694E79400271127F2
:1069F00020E240E063E08AE00E9487068EE20E9487
:106A0000420A80912D0390912E0380FF02C085E3FE
:106A100001C080E30E94420A90912F03892F807663
:106A200009F0C0C397FFBEC39F7790932F0363E025
:106A30008AE00E94860A8FE892E0E9C18F7780930E
:106A4000E20290914E0397FF31C0892F807671F159
:106A50009F7790934E0363E08CE00E94860AE0905B
:106A60004F03FF240027112720E240E062E08AE084
:106A70000E9487068AE30E94420AE0905003FF24A6
:106A80000027112720E340E062E08AE00E948706A9
:106A90008AE30E94420AE0905103FF240027112755
:106AA00020E340E062E08AE00E948706909128039C
:106AB00097FF35C0892F807691F19F7790932803B7
:106AC00060E080E00E94860A88E892E00E94620A04
:106AD00080912603909127036AE070E00E94F439C8
:106AE000882799277B018C0120E340E062E08AE05F
:106AF0000E9487068EE20E94420A809126039091AE
:106B000027036AE070E00E94F439AA27BB277C01C2
:106B10008D0120E340E061E08AE00E9487069091C9
:106B20002803892F807661F497FF0AC09F7790939E
:106B3000280360E00E94860A8DE792E00E94620AC4
:106B40009091EA0297FF35C0892F807691F19F7767
:106B50009093EA0260E08AE00E94860A86E792E06B
:106B60000E94620A8091E8029091E9026AE070E076
:106B70000E94F439882799277B018C0120E340E0AB
:106B800062E08AE00E9487068EE20E94420A8091BB
:106B9000E8029091E9026AE070E00E94F439AA27C5
:106BA000BB277C018D0120E340E061E08AE00E9488
:106BB00087069091EA02892F807669F497FF0BC0CF
:106BC0009F779093EA0260E08AE00E94860A8BE653
:106BD00092E00E94620A90911E0397FF1AC0892FCB
:106BE0008076B9F09F7790931E0361E080E00E9469
:106BF000860A85E692E00E94620AE0901C03F0900B
:106C00001D030027112720E240E063E08AE00E9494
:106C1000870690911E03892F807661F497FF0AC042
:106C20009F7790931E0361E00E94860A8CE592E0B4
:106C30000E94620A9091070397FF35C0892F8076E2
:106C400091F19F779093070361E08BE00E94860AA1
:106C500087E592E00E94620A809105039091060305
:106C60006AE070E00E94F439882799277B018C0143
:106C700020E240E063E08AE00E9487068EE20E9404
:106C8000420A80910503909106036AE070E00E9439
:106C9000F439AA27BB277C018D0120E340E061E0A5
:106CA0008AE00E94870690910703892F807669F415
:106CB00097FF0BC09F779093070361E08BE00E94E2
:106CC000860A8DE492E00E94620A90913B0397FF4E
:106CD0003DC0892F8076D1F19F7790933B0362E08E
:106CE00080E00E94860A87E492E00E94620A609136
:106CF0003703709138038091390390913A0324E669
:106D000030E040E050E00E941B3A79018A0120E225
:106D100040E064E08AE00E9487068EE20E94420A18
:106D200060913703709138038091390390913A0351
:106D300024E630E040E050E00E941B3A7B018C01E9
:106D400020E340E062E08AE00E94870690913B03E6
:106D5000892F807661F497FF0AC09F7790933B0359
:106D600062E00E94860A8AE392E00E94620A9091A1
:106D7000400397FF3DC0892F8076D1F19F77909394
:106D8000400363E080E00E94860A84E392E00E9470
:106D9000620A60913C0370913D0380913E039091A3
:106DA0003F032AE030E040E050E00E941B3A7901C6
:106DB0008A0120E240E064E08AE00E9487068EE2D9
:106DC0000E94420A60913C0370913D0380913E0312
:106DD00090913F032AE030E040E050E00E941B3AEF
:106DE0007B018C0120E340E061E08AE00E9487069D
:106DF00090914003892F807609F0D4C197FFD2C1CA
:106E00009F779093400363E00E94860AC1010E942D
:106E1000620AC8C18F778093E2029091760397FF50
:106E200026C0892F807619F19F779093760360E0D2
:106E300080E00E94860A8AE192E00E94620A60E095
:106E400085E00E94860A8EE593E00E94550A60E084
:106E50008CE00E94860A81E192E00E94620A60E072
:106E60008FE00E94860A84E693E00E94550A909182
:106E70000C0397FF35C0892F807691F19F7790930F
:106E80000C0361E080E00E94860A8CE092E00E94A0
:106E9000620A80910A0390910B0364E670E00E94FD
:106EA000F439882799277B018C0120E240E062E0D9
:106EB0008AE00E9487068EE20E94420A80910A03BD
:106EC00090910B0364E670E00E94F439AA27BB2777
:106ED0007C018D0120E340E062E08AE00E948706A9
:106EE00090910C03892F807661F497FF0AC09F77F9
:106EF00090930C0361E00E94860A82E092E00E9477
:106F0000620A9091180397FF35C0892F807691F11E
:106F10009F779093180361E08BE00E94860A8DEFC3
:106F200091E00E94620A80911603909117036AE033
:106F300070E00E94F439882799277B018C0120E2B8
:106F400040E063E08AE00E9487068EE20E94420AE7
:106F500080911603909117036AE070E00E94F43963
:106F6000AA27BB277C018D0120E340E061E08AE095
:106F70000E94870690911803892F807669F497FF05
:106F80000BC09F779093180361E08BE00E94860A04
:106F900083EF91E00E94620A9091070397FF35C04A
:106FA000892F807691F19F779093070362E08BE0C1
:106FB0000E94860A8EEE91E00E94620A809105038B
:106FC000909106036AE070E00E94F43988279927BF
:106FD0007B018C0120E240E063E08AE00E948706AA
:106FE0008EE20E94420A80910503909106036AE0B6
:106FF00070E00E94F439AA27BB277C018D0120E3B1
:1070000040E061E08AE00E94870690910703892FA3
:10701000807669F497FF0BC09F779093070362E037
:107020008BE00E94860A84EE91E00E94620A9091B1
:10703000130397FF3DC0892F8076D1F19F779093FE
:10704000130362E080E00E94860A8FED91E00E94C7
:10705000620A60910F037091100380911103909167
:10706000120324E630E040E050E00E941B3A790130
:107070008A0120E240E063E08AE00E9487068EE217
:107080000E94420A60910F037091100380911103D6
:107090009091120324E630E040E050E00E941B3A59
:1070A0007B018C0120E340E062E08AE00E948706D9
:1070B00090911303892F807661F497FF0AC09F7720
:1070C0009093130362E00E94860A85ED91E00E948E
:1070D000620A90916B0397FF65C0892F807609F44F
:1070E00061C09F7790936B0363E080E00E94860A03
:1070F000809172030E94420AE0906A03FF240027F5
:10710000112720E340E062E08AE00E9487068DE2DA
:107110000E94420AE0906C03FF240027112720E31D
:1071200040E062E08AE00E9487068EE20E94420A06
:10713000E0906D03FF240027112720E340E062E088
:107140008AE00E94870663E08AE00E94860A8091B6
:1071500073030E94420AE0906E03FF240027112768
:1071600020E340E063E08AE00E9487068DE20E940F
:10717000420AE0907003FF240027112720E340E03B
:1071800062E08AE00E9487068EE20E94420AE09056
:107190007103FF240027112720E340E062E08AE02A
:1071A0000E9487060E948A2E813029F0823011F0D9
:1071B0000C94DA2F0FC0809102028F5F809302023D
:1071C000833010F0109202020E94750A0E94112E64
:1071D0000C94DA2F879B07C080E00E94D108979813
:1071E00010922B0307C08FEF0E94D108979A8CE072
:1071F00080932B0380912C03806180932C038091DA
:10720000E20280618093E2020C94DA2FFC0188276D
:107210009927E89421912032E9F3293010F02E309B
:10722000C8F32B3241F02D3239F4689404C00E9427
:107230009139820F911D219120532A30C0F31EF401
:10724000909581959F4F08951F93FC01992788275A
:10725000BC01E89411911032E9F3193010F01E309E
:10726000C8F31B3251F01D3249F4689406C00E94E5
:107270007C39610F711D811D911D119110531A30C0
:10728000B0F33EF490958095709561957F4F8F4F48
:107290009F4F1F9108950C94583AFB01DC0102C0E6
:1072A00005900D9241505040D8F70895FB01DC0144
:1072B00005900D920020E1F70895FB01DC0141509B
:1072C000504030F08D910590801919F40020B9F7E5
:1072D000881B990B0895FB01DC0101900D920020A1
:1072E000E1F70895DC016C9161566A3108F0605E47
:1072F0006F5B6D93C1F70895592F482F372F262FB5
:10730000660F771F881F991F660F771F881F991FA9
:10731000620F731F841F951F660F771F881F991FA9
:1073200008957AE0979F902D879F802D910D1124CD
:107330000895803239F0992329F480321CF08F3778
:107340000CF4089523C0E199FECFBFBBAEBBE09A19
:1073500011960DB20895F7DF01921A94E1F708959E
:10736000F2DFE02DF0DFF02D0895E199FECFBFBBF5
:10737000AEBB0DBA11960FB6F894E29AE19A0FBE21
:107380000895F3DF012CF1DF112408959927882750
:107390000895629FD001739FF001829FE00DF11D5F
:1073A000649FE00DF11D929FF00D839FF00D749F7F
:1073B000F00D659FF00D9927729FB00DE11DF91F2B
:1073C000639FB00DE11DF91FBD01CF011124089588
:1073D000991B79E004C0991F961708F0961B881F27
:1073E0007A95C9F780950895AA1BBB1B51E107C088
:1073F000AA1FBB1FA617B70710F0A61BB70B881F45
:10740000991F5A95A9F780959095BC01CD010895D3
:1074100097FB092E07260AD077FD04D0E5DF06D0BA
:1074200000201AF4709561957F4F0895F6F79095B6
:1074300081959F4F0895A1E21A2EAA1BBB1BFD0147
:107440000DC0AA1FBB1FEE1FFF1FA217B307E40743
:10745000F50720F0A21BB30BE40BF50B661F771F9B
:10746000881F991F1A9469F760957095809590957B
:107470009B01AC01BD01CF01089597FB092E0526A4
:107480000ED057FD04D0D7DF0AD0001C38F4509539
:107490004095309521953F4F4F4F5F4F0895F6F738
:1074A00090958095709561957F4F8F4F9F4F089570
:0274B000FFCF0C
:0474B20001FFFF00D7
:00000001FF
